******************************************************************************
               TMS320C6x Linker PC v7.4.2                      
******************************************************************************
>> Linked Tue Sep 30 08:27:08 2014

OUTPUT FILE NAME:   <EMACLoopback_testProject.out>
ENTRY POINT SYMBOL: "_c_int00"  address: 0084ad40


MEMORY CONFIGURATION

         name            origin    length      used     unused   attr    fill
----------------------  --------  ---------  --------  --------  ----  --------
  L2SRAM                00800000   00100000  0005ff48  000a00b8  RW X
  MSMCSRAM              0c000000   00100000  00000000  00100000  RW X
  DDR3                  80000000   20000000  00000da0  1ffff260  RWIX


SEGMENT ALLOCATION MAP

run origin  load origin   length   init length attrs members
----------  ----------- ---------- ----------- ----- -------
00800000    00800000    00030000   00000000    rw-
  00800000    00800000    00030000   00000000    rw- .far:PKTBUF_L2MEM
00830000    00830000    0001ef80   0001ef80    r-x
  00830000    00830000    0001ef80   0001ef80    r-x .text
0084ef80    0084ef80    00008000   00000000    rw-
  0084ef80    0084ef80    00008000   00000000    rw- systemHeapMaster
00856f80    00856f80    00003102   00003102    r--
  00856f80    00856f80    00003102   00003102    r-- .const
0085a088    0085a088    000032d4   00000000    rw-
  0085a088    0085a088    000032d4   00000000    rw- .far
0085d360    0085d360    00001000   00000000    rw-
  0085d360    0085d360    00001000   00000000    rw- .stack
0085e360    0085e360    000008fc   000008fc    rw-
  0085e360    0085e360    000008fc   000008fc    rw- .fardata
0085ec60    0085ec60    00000800   00000000    rw-
  0085ec60    0085ec60    00000800   00000000    rw- .far:taskStackSection
0085f460    0085f460    00000014   00000014    r--
  0085f460    0085f460    00000014   00000014    r-- .switch.1
0085f480    0085f480    000002b4   00000000    rw-
  0085f480    0085f480    00000194   00000000    rw- emacComm
  0085f614    0085f614    00000120   00000000    rw- .cio
0085f734    0085f734    00000070   00000070    r--
  0085f734    0085f734    00000070   00000070    r-- .switch.2
0085f7a4    0085f7a4    00000008   00000000    rw-
  0085f7a4    0085f7a4    00000008   00000000    rw- .bss
0085f7ac    0085f7ac    00000012   00000012    rw-
  0085f7ac    0085f7ac    00000012   00000012    rw- .neardata
0085f800    0085f800    000007a4   000007a4    r-x
  0085f800    0085f800    00000200   00000200    r-x .vecs
  0085fa00    0085fa00    000005a4   000005a4    r-- .cinit
80000000    80000000    00000da0   00000da0    rw-
  80000000    80000000    00000da0   00000da0    rw- platform_lib


SECTION ALLOCATION MAP

 output                                  attributes/
section   page    origin      length       input sections
--------  ----  ----------  ----------   ----------------
.init_array 
*          0    00800000    00000000     UNINITIALIZED

xdc.meta   0    00800000    00000120     COPY SECTION
                  00800000    00000120     evmc6657_pe66.oe66 (xdc.meta)

.far:PKTBUF_L2MEM 
*          0    00800000    00030000     UNINITIALIZED
                  00800000    00030000     my_test_main.obj (.far:PKTBUF_L2MEM)

.text      0    00830000    0001ef80     
                  00830000    00001ea0     ti.platform.evm6657l.ae66 : platform.obj (.text)
                  00831ea0    00001900                               : evmc6657.obj (.text)
                  008337a0    00001740     my_test_main.obj (.text)
                  00834ee0    000010c0     ti.platform.evm6657l.ae66 : evmc665x_nand.obj (.text)
                  00835fa0    00000d80                               : evmc665x_i2c_eeprom.obj (.text)
                  00836d20    000009a0     ti.targets.rts6000.ae66 : System.oe66 (.text:xdc_runtime_System_doPrint__I)
                  008376c0    000007e0     ti.drv.emac.ae66 : emac.oe66 (.text:EMAC_coreInit)
                  00837ea0    00000780     sysbios.lib : BIOS.obj (.text:ti_sysbios_family_c64p_Exception_handler__I)
                  00838620    00000700     ti.drv.emac.ae66 : mdio.oe66 (.text:MDIO_timerTick)
                  00838d20    000006c0     ti.platform.evm6657l.ae66 : evmc665x_uart.obj (.text)
                  008393e0    00000660     ti.drv.emac.ae66 : emac_drv.oe66 (.text:emac_init)
                  00839a40    00000660     sysbios.lib : BIOS.obj (.text:ti_sysbios_heaps_HeapMem_free__E)
                  0083a0a0    00000620                 : BIOS.obj (.text:ti_sysbios_heaps_HeapMem_alloc__E)
                  0083a6c0    000005e0     ti.drv.emac.ae66 : emac_drv.oe66 (.text:emac_open)
                  0083aca0    000005c0     rts6600_elf.lib : divd.obj (.text:__c6xabi_divd)
                  0083b260    000005c0                     : _printfi.obj (.text:_getarg_diouxp)
                  0083b820    000005c0     ti.platform.evm6657l.ae66 : evmc665x_spi.obj (.text)
                  0083bde0    000005c0     sysbios.lib : BIOS.obj (.text:ti_sysbios_timers_timer64_Timer_Module_startup__F)
                  0083c3a0    00000560     ti.drv.emac.ae66 : emac.oe66 (.text:EMAC_commonInit)
                  0083c900    00000520     ti.platform.evm6657l.ae66 : evmc665x_nor.obj (.text)
                  0083ce20    00000500     sysbios.lib : BIOS.obj (.text:ti_sysbios_knl_Task_Instance_finalize__F)
                  0083d320    000004c0     ti.platform.evm6657l.ae66 : evmc665x_fpga.obj (.text)
                  0083d7e0    00000460     rts6600_elf.lib : _printfi.obj (.text:_printfi)
                  0083dc40    00000460                     : _printfi.obj (.text:_setfield)
                  0083e0a0    00000400     sysbios.lib : BIOS.obj (.text:ti_sysbios_knl_Semaphore_pend__E)
                  0083e4a0    000003e0     ti.drv.emac.ae66 : emac.oe66 (.text:EMAC_coreDeInit)
                  0083e880    000003c0     sysbios.lib : BIOS.obj (.text:ti_sysbios_knl_Task_Instance_init__F)
                  0083ec40    000003a0     rts6600_elf.lib : fputs.obj (.text:fputs)
                  0083efe0    00000360     evmc6657_pe66.oe66 (.text:xdc_runtime_System_printfExtend__I)
                  0083f340    00000320     rts6600_elf.lib : _printfi.obj (.text:_pproc_fge)
                  0083f660    00000320     my_test_osal.obj (.text)
                  0083f980    00000300     ti.drv.emac.ae66 : emac_drv.oe66 (.text:emac_poll)
                  0083fc80    00000300     sysbios.lib : BIOS.obj (.text:ti_sysbios_family_c64p_Hwi_dispatchC__I)
                  0083ff80    000002e0     rts6600_elf.lib : _printfi.obj (.text:_pproc_fwp)
                  00840260    000002e0     sysbios.lib : BIOS.obj (.text:ti_sysbios_knl_Task_Module_startup__F)
                  00840540    000002a0     rts6600_elf.lib : _printfi.obj (.text:fcvt)
                  008407e0    000002a0     sysbios.lib : BIOS.obj (.text:ti_sysbios_knl_Clock_workFunc__E)
                  00840a80    00000280                 : BIOS.obj (.text:deviceConfig$44)
                  00840d00    00000280     rts6600_elf.lib : _printfi.obj (.text:ecvt)
                  00840f80    00000280     ti.drv.emac.ae66 : emac_drv.oe66 (.text:emac_config)
                  00841200    00000280     sysbios.lib : BIOS.obj (.text:ti_sysbios_knl_Clock_Instance_init__F)
                  00841480    00000280                 : BIOS.obj (.text:ti_sysbios_knl_Task_exit__E)
                  00841700    00000280     ti.targets.rts6000.ae66 : Core-mem.oe66 (.text:xdc_runtime_Core_createObject__I)
                  00841980    00000280                             : Error.oe66 (.text:xdc_runtime_Error_raiseX__F)
                  00841c00    00000260     ti.drv.emac.ae66 : emac.oe66 (.text:EMAC_setMulticast)
                  00841e60    00000260                      : emac_drv.oe66 (.text:emac_send)
                  008420c0    00000260     ti.targets.rts6000.ae66 : Startup.oe66 (.text:xdc_runtime_Startup_startMods__I)
                  00842320    00000240     rts6600_elf.lib : imath64.obj (.text:__c6xabi_divull)
                  00842560    00000240                     : _printfi.obj (.text:_pconv_e)
                  008427a0    00000240                     : _printfi.obj (.text:_pproc_diouxp)
                  008429e0    00000240     sysbios.lib : BIOS.obj (.text:ti_sysbios_family_c64p_Exception_internalHandler__I)
                  00842c20    00000240                 : BIOS.obj (.text:ti_sysbios_knl_Semaphore_post__E)
                  00842e60    00000220     ti.drv.emac.ae66 : emac.oe66 (.text:EMAC_sendPacket)
                  00843080    00000220     rts6600_elf.lib : _printfi.obj (.text:_pproc_str)
                  008432a0    00000220                     : fputc.obj (.text:fputc)
                  008434c0    00000220     sysbios.lib : BIOS.obj (.text:ti_sysbios_family_c64p_Hwi_reconfig__E)
                  008436e0    00000220                 : BIOS.obj (.text:ti_sysbios_knl_Swi_run__I)
                  00843900    00000220                 : BIOS.obj (.text:ti_sysbios_knl_Task_schedule__I)
                  00843b20    00000220                 : BIOS.obj (.text:ti_sysbios_knl_Task_startup__E)
                  00843d40    00000200     ti.drv.emac.ae66 : emac.oe66 (.text:EMAC_RxServiceCheck)
                  00843f40    00000200     rts6600_elf.lib : _printfi.obj (.text:_pconv_g)
                  00844140    00000200     sysbios.lib : c64p_Hwi_disp_always.obj (.text:_ti_sysbios_family_c64p_Hwi_dispatchAlways)
                  00844340    00000200                 : BIOS.obj (.text:block$56)
                  00844540    00000200     rts6600_elf.lib : setvbuf.obj (.text:setvbuf)
                  00844740    000001e0     ti.drv.emac.ae66 : sgmii.oe66 (.text:SGMII_config)
                  00844920    000001e0                      : emac.oe66 (.text:emacDequeueRx)
                  00844b00    000001e0     sysbios.lib : BIOS.obj (.text:ti_sysbios_knl_Task_postInit__I)
                  00844ce0    000001e0                 : BIOS.obj (.text:ti_sysbios_timers_timer64_Timer_getFreq__E)
                  00844ec0    000001c0     ti.drv.emac.ae66 : emac.oe66 (.text:EMAC_TxServiceCheck)
                  00845080    000001c0     rts6600_elf.lib : _printfi.obj (.text:_mcpy)
                  00845240    000001c0     sysbios.lib : BIOS.obj (.text:ti_sysbios_knl_Task_checkStacks__E)
                  00845400    000001c0                 : BIOS.obj (.text:ti_sysbios_timers_timer64_Timer_setPeriodMicroSecs__E)
                  008455c0    000001a0     rts6600_elf.lib : trgdrv.obj (.text:HOSTrename)
                  00845760    000001a0                     : imath40.obj (.text:__c6xabi_divul)
                  00845900    000001a0     ti.drv.emac.ae66 : emac_drv.oe66 (.text:emac_init_queue)
                  00845aa0    000001a0     sysbios.lib : BIOS.obj (.text:ti_sysbios_gates_GateMutex_enter__E)
                  00845c40    000001a0                 : BIOS.obj (.text:ti_sysbios_timers_timer64_Timer_start__E)
                  00845de0    00000180     ti.drv.emac.ae66 : emac.oe66 (.text:EMAC_setReceiveFilter)
                  00845f60    00000180     rts6600_elf.lib : copy_decompress_rle.obj (.text:__TI_decompress_rle_core)
                  008460e0    00000180     ti.drv.emac.ae66 : emac.oe66 (.text:emacEnqueueTx)
                  00846260    00000180                      : emac_drv.oe66 (.text:emac_int_service)
                  008463e0    00000180                      : emac_drv.oe66 (.text:emac_rx_packet)
                  00846560    00000180     sysbios.lib : c64p_Exception_asm.obj (.text)
                  008466e0    00000180                 : BIOS.obj (.text:ti_sysbios_heaps_HeapMem_Instance_init__F)
                  00846860    00000180                 : BIOS.obj (.text:ti_sysbios_knl_Swi_schedule__I)
                  008469e0    00000180                 : BIOS.obj (.text:ti_sysbios_knl_Task_unblockI__E)
                  00846b60    00000180     ti.targets.rts6000.ae66 : Text.oe66 (.text:xdc_runtime_Text_putSite__F)
                  00846ce0    00000160     ti.platform.evm6657l.ae66 : evmc665x_phy.obj (.text)
                  00846e40    00000140     ti.csl.ae66 : csl_chip.oe66 (.text:CSL_chipReadReg)
                  00846f80    00000140     boot.ae66 : autoinit.oe66 (.text:_auto_init_elf)
                  008470c0    00000140     rts6600_elf.lib : _printfi.obj (.text:_pproc_fflags)
                  00847200    00000140     ti.drv.emac.ae66 : emac.oe66 (.text:emacDequeueTx)
                  00847340    00000140                      : emac.oe66 (.text:emacEnqueueRx)
                  00847480    00000140     rts6600_elf.lib : lowlev.obj (.text:getdevice)
                  008475c0    00000140     sysbios.lib : BIOS.obj (.text:ti_sysbios_family_c64p_Hwi_Module_startup__F)
                  00847700    00000140                 : BIOS.obj (.text:ti_sysbios_family_c66_Cache_Module_startup__F)
                  00847840    00000140                 : BIOS.obj (.text:ti_sysbios_knl_Clock_Instance_finalize__F)
                  00847980    00000140                 : BIOS.obj (.text:ti_sysbios_knl_Semaphore_Instance_init__F)
                  00847ac0    00000140                 : BIOS.obj (.text:ti_sysbios_knl_Swi_post__E)
                  00847c00    00000140                 : BIOS.obj (.text:ti_sysbios_knl_Task_blockI__E)
                  00847d40    00000120     rts6600_elf.lib : fclose.obj (.text:_closefile)
                  00847e60    00000120                     : _printfi.obj (.text:_ltostr)
                  00847f80    00000120                     : fseek.obj (.text:fseek)
                  008480a0    00000120     sysbios.lib : BIOS.obj (.text:rtsUnlock$0)
                  008481c0    00000120     ti.targets.rts6000.ae66 : Text.oe66 (.text:xdc_runtime_Text_putLab__F)
                  008482e0    00000100     rts6600_elf.lib : trgdrv.obj (.text:HOSTlseek)
                  008483e0    00000100                     : _io_perm.obj (.text:_wrt_ok)
                  008484e0    00000100     ti.drv.emac.ae66 : emac_drv.oe66 (.text:emac_free_chan_comm_pcb)
                  008485e0    00000100                      : emac_drv.oe66 (.text:emac_reset_queue)
                  008486e0    00000100     sysbios.lib : BIOS.obj (.text:initDevice$44)
                  008487e0    00000100                 : BIOS.obj (.text:ti_sysbios_knl_Clock_startI__E)
                  008488e0    00000100                 : BIOS.obj (.text:ti_sysbios_knl_Swi_restoreHwi__E)
                  008489e0    00000100     ti.targets.rts6000.ae66 : Core-mem.oe66 (.text:xdc_runtime_Core_deleteObject__I)
                  00848ae0    00000100                             : Startup.oe66 (.text:xdc_runtime_Startup_exec__F)
                  00848be0    00000100                             : Text.oe66 (.text:xdc_runtime_Text_putMod__F)
                  00848ce0    00000100                             : Text.oe66 (.text:xdc_runtime_Text_visitRope2__I)
                  00848de0    000000e0     rts6600_elf.lib : trgdrv.obj (.text:HOSTopen)
                  00848ec0    000000e0     ti.drv.emac.ae66 : mdio.oe66 (.text:PHYREG_waitResultsAck)
                  00848fa0    000000e0     rts6600_elf.lib : _printfi.obj (.text:_div)
                  00849080    000000e0                     : atoi.obj (.text:atoi)
                  00849160    000000e0                     : lowlev.obj (.text:close)
                  00849240    000000e0                     : copy_zero_init.obj (.text:decompress:ZI:__TI_zero_init)
                  00849320    000000e0     ti.drv.emac.ae66 : emac_drv.oe66 (.text:emac_free_packet)
                  00849400    000000e0                      : emac_drv.oe66 (.text:emac_get_packet)
                  008494e0    000000e0     rts6600_elf.lib : fflush.obj (.text:fflush)
                  008495c0    000000e0                     : ltoa.obj (.text:ltoa)
                  008496a0    000000e0                     : memset.obj (.text:memset)
                  00849780    000000e0                     : printf.obj (.text:printf)
                  00849860    000000e0     sysbios.lib : BIOS.obj (.text:ti_sysbios_family_c64p_Hwi_Instance_finalize__F)
                  00849940    000000e0                 : BIOS.obj (.text:ti_sysbios_family_c64p_Hwi_Instance_init__F)
                  00849a20    000000e0     evmc6657_pe66.oe66 (.text:ti_sysbios_family_c64p_Hwi_Object__create__S)
                  00849b00    000000e0     evmc6657_pe66.oe66 (.text:ti_sysbios_hal_Hwi_Object__create__S)
                  00849be0    000000e0     sysbios.lib : BIOS.obj (.text:ti_sysbios_knl_Clock_start__E)
                  00849cc0    000000e0                 : BIOS.obj (.text:ti_sysbios_timers_timer64_Timer_startup__E)
                  00849da0    000000e0     ti.targets.rts6000.ae66 : Error.oe66 (.text:xdc_runtime_Error_print__F)
                  00849e80    000000e0                             : Memory.oe66 (.text:xdc_runtime_Memory_alloc__F)
                  00849f60    000000c0     rts6600_elf.lib : trgdrv.obj (.text:HOSTread)
                  0084a020    000000c0                     : trgdrv.obj (.text:HOSTunlink)
                  0084a0e0    000000c0                     : trgdrv.obj (.text:HOSTwrite)
                  0084a1a0    000000c0     ti.drv.emac.ae66 : mdio.oe66 (.text:PHYREG_waitResults)
                  0084a260    000000c0     rts6600_elf.lib : dtor_list.obj (.text:_Z11__TI_atexitPFYvPvES_S_)
                  0084a320    000000c0                     : dtor_list.obj (.text:__cxa_finalize)
                  0084a3e0    000000c0                     : divu.obj (.text:__divu)
                  0084a4a0    000000c0                     : fflush.obj (.text:_doflush)
                  0084a560    000000c0     ti.drv.emac.ae66 : emac_drv.oe66 (.text:emac_status_update)
                  0084a620    000000c0     rts6600_elf.lib : exit.obj (.text:exit)
                  0084a6e0    000000c0     sysbios.lib : BIOS.obj (.text:ti_sysbios_BIOS_errorRaiseHook__I)
                  0084a7a0    000000c0                 : BIOS.obj (.text:ti_sysbios_heaps_HeapMem_getStats__E)
                  0084a860    000000c0                 : BIOS.obj (.text:ti_sysbios_knl_Clock_logTick__E)
                  0084a920    000000c0     evmc6657_pe66.oe66 (.text:ti_sysbios_knl_Task_Object__create__S)
                  0084a9e0    000000c0     sysbios.lib : BIOS.obj (.text:ti_sysbios_timers_timer64_Timer_stop__E)
                  0084aaa0    000000c0     ti.targets.rts6000.ae66 : System.oe66 (.text:xdc_runtime_System_formatNum__I)
                  0084ab60    000000a0     rts6600_elf.lib : trgdrv.obj (.text:HOSTclose)
                  0084ac00    000000a0     ti.drv.emac.ae66 : mdio.oe66 (.text:PHYREG_wait)
                  0084aca0    000000a0     rts6600_elf.lib : remu.obj (.text:__remu)
                  0084ad40    000000a0     boot.ae66 : boot.oe66 (.text:_c_int00)
                  0084ade0    000000a0     rts6600_elf.lib : fopen.obj (.text:_cleanup)
                  0084ae80    000000a0                     : _printfi.obj (.text:_ecpy)
                  0084af20    000000a0                     : _printfi.obj (.text:_fcpy)
                  0084afc0    000000a0                     : _printfi.obj (.text:_pconv_f)
                  0084b060    000000a0     sysbios.lib : c64p_Hwi_asm.obj (.text:_ti_sysbios_family_c64p_Hwi_plug__E)
                  0084b100    000000a0     ti.drv.emac.ae66 : emac_drv.oe66 (.text:emac_free_macaddr)
                  0084b1a0    000000a0                      : emac_drv.oe66 (.text:emac_queue_pop)
                  0084b240    000000a0     rts6600_elf.lib : lowlev.obj (.text:finddevice)
                  0084b2e0    000000a0                     : lowlev.obj (.text:lseek)
                  0084b380    000000a0                     : memcpy64.obj (.text:memcpy)
                  0084b420    000000a0     sysbios.lib : BIOS.obj (.text:ti_sysbios_heaps_HeapMem_init__I)
                  0084b4c0    000000a0     rts6600_elf.lib : lowlev.obj (.text:write)
                  0084b560    000000a0     ti.targets.rts6000.ae66 : Assert.oe66 (.text:xdc_runtime_Assert_raise__I)
                  0084b600    00000080     ti.drv.emac.ae66 : mdio.oe66 (.text:MDIO_open)
                  0084b680    00000080     rts6600_elf.lib : llshift.obj (.text:__c6xabi_llshl)
                  0084b700    00000080     sysbios.lib : c62_TaskSupport_asm.obj (.text:_ti_sysbios_family_c62_TaskSupport_swap__E)
                  0084b780    00000080     ti.drv.emac.ae66 : emac_drv.oe66 (.text:emac_statistics_update)
                  0084b800    00000080     evmc6657_pe66.oe66 (.text:malloc)
                  0084b880    00000080     rts6600_elf.lib : trgmsg.obj (.text:readmsg)
                  0084b900    00000080                     : strncpy.obj (.text:strncpy)
                  0084b980    00000080     ti.platform.evm6657l.ae66 : evm665x_i2c.obj (.text)
                  0084ba00    00000080     sysbios.lib : BIOS.obj (.text:ti_sysbios_family_c62_TaskSupport_start__E)
                  0084ba80    00000080                 : BIOS.obj (.text:ti_sysbios_family_c64p_Exception_Module_startup__F)
                  0084bb00    00000080                 : BIOS.obj (.text:ti_sysbios_family_c64p_Hwi_eventMap__E)
                  0084bb80    00000080                 : BIOS.obj (.text:ti_sysbios_family_c66_Cache_invL1pAll__E)
                  0084bc00    00000080     evmc6657_pe66.oe66 (.text:ti_sysbios_gates_GateHwi_Object__create__S)
                  0084bc80    00000080     evmc6657_pe66.oe66 (.text:ti_sysbios_gates_GateMutex_Object__create__S)
                  0084bd00    00000080     sysbios.lib : BIOS.obj (.text:ti_sysbios_hal_Hwi_checkStack:ti_sysbios_hal_Hwi_checkStack)
                  0084bd80    00000080     evmc6657_pe66.oe66 (.text:ti_sysbios_heaps_HeapMem_Object__create__S)
                  0084be00    00000080     sysbios.lib : BIOS.obj (.text:ti_sysbios_knl_Clock_Module_startup__F)
                  0084be80    00000080     evmc6657_pe66.oe66 (.text:ti_sysbios_knl_Clock_Object__create__S)
                  0084bf00    00000080     sysbios.lib : BIOS.obj (.text:ti_sysbios_knl_Clock_getTicks__E)
                  0084bf80    00000080                 : BIOS.obj (.text:ti_sysbios_knl_Idle_loop__E)
                  0084c000    00000080     evmc6657_pe66.oe66 (.text:ti_sysbios_knl_Queue_Object__create__S)
                  0084c080    00000080     evmc6657_pe66.oe66 (.text:ti_sysbios_knl_Semaphore_Object__create__S)
                  0084c100    00000080     sysbios.lib : BIOS.obj (.text:ti_sysbios_knl_Semaphore_pendTimeout__I)
                  0084c180    00000080                 : BIOS.obj (.text:ti_sysbios_knl_Swi_startup__E)
                  0084c200    00000080                 : BIOS.obj (.text:ti_sysbios_knl_Task_restore__E)
                  0084c280    00000080                 : BIOS.obj (.text:ti_sysbios_timers_timer64_Timer_getCount__E)
                  0084c300    00000080                 : BIOS.obj (.text:ti_sysbios_timers_timer64_Timer_getPeriod__E)
                  0084c380    00000080     rts6600_elf.lib : lowlev.obj (.text:unlink)
                  0084c400    00000080     ti.targets.rts6000.ae66 : Core-label.oe66 (.text:xdc_runtime_Core_assignLabel__I)
                  0084c480    00000080                             : Core-params.oe66 (.text:xdc_runtime_Core_assignParams__I)
                  0084c500    00000080                             : System.oe66 (.text:xdc_runtime_System_atexit__F)
                  0084c580    00000080                             : System.oe66 (.text:xdc_runtime_System_rtsExit__I)
                  0084c600    00000080                             : Text.oe66 (.text:xdc_runtime_Text_printVisFxn__I)
                  0084c680    00000080                             : Text.oe66 (.text:xdc_runtime_Text_xprintf__I)
                  0084c700    00000060     ti.drv.emac.ae66 : mdio.oe66 (.text:PHYREG_write)
                  0084c760    00000060                      : sgmii.oe66 (.text:SGMII_reset)
                  0084c7c0    00000060     rts6600_elf.lib : frcmpyd_div.obj (.text:__c6xabi_frcmpyd_div)
                  0084c820    00000060                     : llshift.obj (.text:__c6xabi_llshru)
                  0084c880    00000060                     : imath64.obj (.text:_subcull)
                  0084c8e0    00000060     ti.drv.emac.ae66 : emac_drv.oe66 (.text:emac_queue_push)
                  0084c940    00000060                      : emac_drv.oe66 (.text:emac_reset)
                  0084c9a0    00000060     rts6600_elf.lib : memccpy.obj (.text:memccpy)
                  0084ca00    00000060                     : strncmp.obj (.text:strncmp)
                  0084ca60    00000060     evmc6657_pe66.oe66 (.text:ti_sysbios_BIOS_exitFunc__I)
                  0084cac0    00000060     sysbios.lib : BIOS.obj (.text:ti_sysbios_BIOS_registerRTSLock__I)
                  0084cb20    00000060                 : BIOS.obj (.text:ti_sysbios_gates_GateMutex_Instance_init__F)
                  0084cb80    00000060                 : BIOS.obj (.text:ti_sysbios_hal_Hwi_Instance_init__F)
                  0084cbe0    00000060                 : BIOS.obj (.text:ti_sysbios_hal_Hwi_initStack:ti_sysbios_hal_Hwi_initStack)
                  0084cc40    00000060     evmc6657_pe66.oe66 (.text:ti_sysbios_heaps_HeapMem_Object__get__S)
                  0084cca0    00000060     evmc6657_pe66.oe66 (.text:ti_sysbios_knl_Clock_doTick__I)
                  0084cd00    00000060     evmc6657_pe66.oe66 (.text:ti_sysbios_knl_Queue_Object__get__S)
                  0084cd60    00000060     sysbios.lib : BIOS.obj (.text:ti_sysbios_knl_Swi_Module_startup__F)
                  0084cdc0    00000060     evmc6657_pe66.oe66 (.text:ti_sysbios_knl_Swi_Object__get__S)
                  0084ce20    00000060     evmc6657_pe66.oe66 (.text:ti_sysbios_knl_Task_Object__get__S)
                  0084ce80    00000060     sysbios.lib : BIOS.obj (.text:ti_sysbios_knl_Task_allBlockedFunction__I)
                  0084cee0    00000060                 : BIOS.obj (.text:ti_sysbios_knl_Task_enter__I)
                  0084cf40    00000060     rts6600_elf.lib : vsprintf.obj (.text:vsprintf)
                  0084cfa0    00000060                     : trgmsg.obj (.text:writemsg)
                  0084d000    00000060     ti.targets.rts6000.ae66 : Memory.oe66 (.text:xdc_runtime_Memory_calloc__F)
                  0084d060    00000060                             : SysStd.oe66 (.text:xdc_runtime_SysStd_abort__F)
                  0084d0c0    00000060                             : System.oe66 (.text:xdc_runtime_System_avprintf__F)
                  0084d120    00000060                             : System.oe66 (.text:xdc_runtime_System_vprintf__F)
                  0084d180    00000060                             : Text.oe66 (.text:xdc_runtime_Text_cordText__F)
                  0084d1e0    00000040     ti.drv.emac.ae66 : mdio.oe66 (.text:PHYREG_read)
                  0084d220    00000040     rts6600_elf.lib : isinf.obj (.text:__c6xabi_isinf)
                  0084d260    00000040                     : _printfi.obj (.text:__c6xabi_isnan)
                  0084d2a0    00000040                     : args_main.obj (.text:_args_main)
                  0084d2e0    00000040                     : vsprintf.obj (.text:_outs)
                  0084d320    00000040     sysbios.lib : c62_TaskSupport_asm.obj (.text:_ti_sysbios_family_c62_TaskSupport_buildTaskStack)
                  0084d360    00000040                 : c64p_Hwi_asm_switch.obj (.text:_ti_sysbios_family_xxx_Hwi_switchToIsrStack)
                  0084d3a0    00000040     ti.drv.emac.ae66 : emac.oe66 (.text:emacUpdateStats)
                  0084d3e0    00000040     evmc6657_pe66.oe66 (.text:free)
                  0084d420    00000040     ti.drv.emac.ae66 : emac.oe66 (.text:pqPop)
                  0084d460    00000040                      : emac.oe66 (.text:pqPush)
                  0084d4a0    00000040                      : emac.oe66 (.text:pqPushChain)
                  0084d4e0    00000040     sysbios.lib : BIOS.obj (.text:rtsLock$0)
                  0084d520    00000040     rts6600_elf.lib : strlen.obj (.text:strlen)
                  0084d560    00000040     evmc6657_pe66.oe66 (.text:ti_sysbios_BIOS_startFunc__I)
                  0084d5a0    00000040     sysbios.lib : BIOS.obj (.text:ti_sysbios_BIOS_start__E)
                  0084d5e0    00000040     evmc6657_pe66.oe66 (.text:ti_sysbios_family_c64p_Hwi_Module__startupDone__F)
                  0084d620    00000040     evmc6657_pe66.oe66 (.text:ti_sysbios_family_c64p_Hwi_Object__delete__S)
                  0084d660    00000040     sysbios.lib : BIOS.obj (.text:ti_sysbios_family_c64p_Hwi_disableInterrupt__E)
                  0084d6a0    00000040                 : BIOS.obj (.text:ti_sysbios_family_c64p_Hwi_enableInterrupt__E)
                  0084d6e0    00000040     evmc6657_pe66.oe66 (.text:ti_sysbios_gates_GateHwi_Handle__label__S)
                  0084d720    00000040     evmc6657_pe66.oe66 (.text:ti_sysbios_gates_GateHwi_Object__delete__S)
                  0084d760    00000040     evmc6657_pe66.oe66 (.text:ti_sysbios_gates_GateMutex_Handle__label__S)
                  0084d7a0    00000040     sysbios.lib : BIOS.obj (.text:ti_sysbios_gates_GateMutex_Instance_finalize__F)
                  0084d7e0    00000040     evmc6657_pe66.oe66 (.text:ti_sysbios_gates_GateMutex_Object__delete__S)
                  0084d820    00000040     sysbios.lib : BIOS.obj (.text:ti_sysbios_gates_GateMutex_leave__E)
                  0084d860    00000040     evmc6657_pe66.oe66 (.text:ti_sysbios_hal_Hwi_HwiProxy_Object__create__S)
                  0084d8a0    00000040     sysbios.lib : BIOS.obj (.text:ti_sysbios_hal_Hwi_Instance_finalize__F)
                  0084d8e0    00000040     evmc6657_pe66.oe66 (.text:ti_sysbios_hal_Hwi_Params__init__S)
                  0084d920    00000040     evmc6657_pe66.oe66 (.text:ti_sysbios_hal_Timer_Module__startupDone__F)
                  0084d960    00000040     evmc6657_pe66.oe66 (.text:ti_sysbios_heaps_HeapMem_Handle__label__S)
                  0084d9a0    00000040     evmc6657_pe66.oe66 (.text:ti_sysbios_heaps_HeapMem_Object__delete__S)
                  0084d9e0    00000040     evmc6657_pe66.oe66 (.text:ti_sysbios_knl_Clock_Object__destruct__S)
                  0084da20    00000040     evmc6657_pe66.oe66 (.text:ti_sysbios_knl_Clock_Params__init__S)
                  0084da60    00000040     evmc6657_pe66.oe66 (.text:ti_sysbios_knl_Queue_Object__destruct__S)
                  0084daa0    00000040     sysbios.lib : BIOS.obj (.text:ti_sysbios_knl_Semaphore_Instance_finalize__F)
                  0084dae0    00000040     evmc6657_pe66.oe66 (.text:ti_sysbios_knl_Semaphore_Object__destruct__S)
                  0084db20    00000040     evmc6657_pe66.oe66 (.text:ti_sysbios_knl_Task_Object__first__S)
                  0084db60    00000040     evmc6657_pe66.oe66 (.text:ti_sysbios_knl_Task_Object__next__S)
                  0084dba0    00000040     evmc6657_pe66.oe66 (.text:ti_sysbios_knl_Task_Params__init__S)
                  0084dbe0    00000040     evmc6657_pe66.oe66 (.text:ti_sysbios_timers_timer64_Timer_Module__startupDone__F)
                  0084dc20    00000040     ti.targets.rts6000.ae66 : Error.oe66 (.text:xdc_runtime_Error_check__F)
                  0084dc60    00000040                             : Error.oe66 (.text:xdc_runtime_Error_init__F)
                  0084dca0    00000040     evmc6657_pe66.oe66 (.text:xdc_runtime_Error_raiseX__E)
                  0084dce0    00000040     ti.targets.rts6000.ae66 : Gate.oe66 (.text:xdc_runtime_Gate_leaveSystem__F)
                  0084dd20    00000040     evmc6657_pe66.oe66 (.text:xdc_runtime_IHeap_alloc)
                  0084dd60    00000040     evmc6657_pe66.oe66 (.text:xdc_runtime_IHeap_free)
                  0084dda0    00000040     ti.targets.rts6000.ae66 : Memory.oe66 (.text:xdc_runtime_Memory_free__F)
                  0084dde0    00000040                             : Registry.oe66 (.text:xdc_runtime_Registry_findById__F)
                  0084de20    00000040     evmc6657_pe66.oe66 (.text:xdc_runtime_Startup_exec__I)
                  0084de60    00000040     ti.targets.rts6000.ae66 : System.oe66 (.text:xdc_runtime_System_abort__F)
                  0084dea0    00000040     evmc6657_pe66.oe66 (.text:xdc_runtime_System_aprintf__E)
                  0084dee0    00000040     evmc6657_pe66.oe66 (.text:xdc_runtime_System_printf__E)
                  0084df20    00000040     ti.targets.rts6000.ae66 : Text.oe66 (.text:xdc_runtime_Text_ropeText__F)
                  0084df60    00000040     evmc6657_pe66.oe66 (.text:xdc_runtime_Text_visitRope__I)
                  0084dfa0    00000020     ti.csl.ae66 : csl_gpioGetBaseAddress.oe66 (.text:CSL_GPIO_open)
                  0084dfc0    00000020     ti.drv.emac.ae66 : mdio.oe66 (.text:MDIO_getStatus)
                  0084dfe0    00000020                      : mdio.oe66 (.text:MDIO_initContinue)
                  0084e000    00000020                      : mdio.oe66 (.text:MDIO_initPHY)
                  0084e020    00000020                      : mdio.oe66 (.text:MDIO_initStateMachine)
                  0084e040    00000020     rts6600_elf.lib : negll.obj (.text:__c6xabi_negll)
                  0084e060    00000020                     : dtor_list.obj (.text:__cxa_atexit)
                  0084e080    00000020                     : dtor_list.obj (.text:__cxa_ia64_exit)
                  0084e0a0    00000020     ti.targets.rts6000.ae66 : xdc_noinit.oe66 (.text:__xdc__init)
                  0084e0c0    00000020     rts6600_elf.lib : _lock.obj (.text:_nop)
                  0084e0e0    00000020                     : printf.obj (.text:_outc)
                  0084e100    00000020                     : vsprintf.obj (.text:_outc)
                  0084e120    00000020                     : printf.obj (.text:_outs)
                  0084e140    00000020                     : _lock.obj (.text:_register_lock)
                  0084e160    00000020                     : _lock.obj (.text:_register_unlock)
                  0084e180    00000020     sysbios.lib : c62_TaskSupport_asm.obj (.text:_ti_sysbios_family_c62_TaskSupport_glue)
                  0084e1a0    00000020                 : c64p_Hwi_asm_switch.obj (.text:_ti_sysbios_family_xxx_Hwi_switchToTaskStack)
                  0084e1c0    00000020     rts6600_elf.lib : exit.obj (.text:abort)
                  0084e1e0    00000020                     : dtor_list.obj (.text:atexit)
                  0084e200    00000020                     : copy_decompress_none.obj (.text:decompress:none:__TI_decompress_none)
                  0084e220    00000020                     : copy_decompress_rle.obj (.text:decompress:rle24:__TI_decompress_rle24)
                  0084e240    00000020     ti.drv.emac.ae66 : emac_drv.oe66 (.text:emac_get_version)
                  0084e260    00000020     sysbios.lib : BIOS.obj (.text:nullFunc$0)
                  0084e280    00000020     rts6600_elf.lib : fputc.obj (.text:putc)
                  0084e2a0    00000020                     : fputc.obj (.text:putchar)
                  0084e2c0    00000020     evmc6657_pe66.oe66 (.text:ti_sysbios_BIOS_RtsGateProxy_enter__E)
                  0084e2e0    00000020     evmc6657_pe66.oe66 (.text:ti_sysbios_BIOS_RtsGateProxy_leave__E)
                  0084e300    00000020     sysbios.lib : BIOS.obj (.text:ti_sysbios_BIOS_setThreadType__E)
                  0084e320    00000020     evmc6657_pe66.oe66 (.text:ti_sysbios_family_c62_TaskSupport_Module__startupDone__S)
                  0084e340    00000020     sysbios.lib : BIOS.obj (.text:ti_sysbios_family_c62_TaskSupport_checkStack__E)
                  0084e360    00000020                 : BIOS.obj (.text:ti_sysbios_family_c62_TaskSupport_getStackAlignment__E)
                  0084e380    00000020     evmc6657_pe66.oe66 (.text:ti_sysbios_family_c64p_Exception_Module_startup__E)
                  0084e3a0    00000020     evmc6657_pe66.oe66 (.text:ti_sysbios_family_c64p_Hwi_Module__startupDone__S)
                  0084e3c0    00000020     evmc6657_pe66.oe66 (.text:ti_sysbios_family_c64p_Hwi_Module_startup__E)
                  0084e3e0    00000020     sysbios.lib : BIOS.obj (.text:ti_sysbios_family_c64p_Hwi_clearInterrupt__E)
                  0084e400    00000020                 : BIOS.obj (.text:ti_sysbios_family_c64p_Hwi_startup__E)
                  0084e420    00000020                 : BIOS.obj (.text:ti_sysbios_family_c64p_Hwi_switchFromBootStack__E)
                  0084e440    00000020                 : BIOS.obj (.text:ti_sysbios_family_c64p_Hwi_unPluggedInterrupt__I)
                  0084e460    00000020                 : BIOS.obj (.text:ti_sysbios_family_c64p_tci6488_TimerSupport_enable__E)
                  0084e480    00000020     evmc6657_pe66.oe66 (.text:ti_sysbios_family_c66_Cache_Module_startup__E)
                  0084e4a0    00000020     sysbios.lib : BIOS.obj (.text:ti_sysbios_family_c66_Cache_wbInv__E)
                  0084e4c0    00000020                 : BIOS.obj (.text:ti_sysbios_gates_GateHwi_Instance_init__F)
                  0084e4e0    00000020                 : BIOS.obj (.text:ti_sysbios_gates_GateHwi_enter__E)
                  0084e500    00000020                 : BIOS.obj (.text:ti_sysbios_gates_GateHwi_leave__E)
                  0084e520    00000020     evmc6657_pe66.oe66 (.text:ti_sysbios_gates_GateHwi_query__E)
                  0084e540    00000020     sysbios.lib : BIOS.obj (.text:ti_sysbios_gates_GateHwi_query__F)
                  0084e560    00000020     evmc6657_pe66.oe66 (.text:ti_sysbios_gates_GateMutex_query__E)
                  0084e580    00000020     sysbios.lib : BIOS.obj (.text:ti_sysbios_gates_GateMutex_query__F)
                  0084e5a0    00000020     evmc6657_pe66.oe66 (.text:ti_sysbios_hal_Hwi_HwiProxy_Module__startupDone__S)
                  0084e5c0    00000020     evmc6657_pe66.oe66 (.text:ti_sysbios_hal_Hwi_HwiProxy_Object__delete__S)
                  0084e5e0    00000020     evmc6657_pe66.oe66 (.text:ti_sysbios_hal_Hwi_HwiProxy_clearInterrupt__E)
                  0084e600    00000020     evmc6657_pe66.oe66 (.text:ti_sysbios_hal_Hwi_HwiProxy_disableInterrupt__E)
                  0084e620    00000020     evmc6657_pe66.oe66 (.text:ti_sysbios_hal_Hwi_HwiProxy_enableInterrupt__E)
                  0084e640    00000020     evmc6657_pe66.oe66 (.text:ti_sysbios_hal_Hwi_HwiProxy_startup__E)
                  0084e660    00000020     evmc6657_pe66.oe66 (.text:ti_sysbios_hal_Hwi_HwiProxy_switchFromBootStack__E)
                  0084e680    00000020     evmc6657_pe66.oe66 (.text:ti_sysbios_hal_Hwi_Module_startup__E)
                  0084e6a0    00000020     sysbios.lib : BIOS.obj (.text:ti_sysbios_hal_Hwi_Module_startup__F)
                  0084e6c0    00000020     evmc6657_pe66.oe66 (.text:ti_sysbios_hal_Timer_Module__startupDone__S)
                  0084e6e0    00000020     evmc6657_pe66.oe66 (.text:ti_sysbios_hal_Timer_Module_startup__E)
                  0084e700    00000020     sysbios.lib : BIOS.obj (.text:ti_sysbios_hal_Timer_Module_startup__F)
                  0084e720    00000020     evmc6657_pe66.oe66 (.text:ti_sysbios_hal_Timer_TimerProxy_Module__startupDone__S)
                  0084e740    00000020     evmc6657_pe66.oe66 (.text:ti_sysbios_hal_Timer_TimerProxy_getExpiredCounts__E)
                  0084e760    00000020     evmc6657_pe66.oe66 (.text:ti_sysbios_hal_Timer_TimerProxy_getPeriod__E)
                  0084e780    00000020     evmc6657_pe66.oe66 (.text:ti_sysbios_hal_Timer_TimerProxy_setNextTick__E)
                  0084e7a0    00000020     evmc6657_pe66.oe66 (.text:ti_sysbios_hal_Timer_TimerProxy_startup__E)
                  0084e7c0    00000020     evmc6657_pe66.oe66 (.text:ti_sysbios_heaps_HeapMem_Module_GateProxy_enter__E)
                  0084e7e0    00000020     evmc6657_pe66.oe66 (.text:ti_sysbios_heaps_HeapMem_Module_GateProxy_leave__E)
                  0084e800    00000020     evmc6657_pe66.oe66 (.text:ti_sysbios_heaps_HeapMem_Module_GateProxy_query__E)
                  0084e820    00000020     sysbios.lib : BIOS.obj (.text:ti_sysbios_heaps_HeapMem_isBlocking__E)
                  0084e840    00000020     evmc6657_pe66.oe66 (.text:ti_sysbios_knl_Clock_Module_State_clockQ)
                  0084e860    00000020     evmc6657_pe66.oe66 (.text:ti_sysbios_knl_Clock_Module_startup__E)
                  0084e880    00000020     sysbios.lib : BIOS.obj (.text:ti_sysbios_knl_Queue_Instance_init__F)
                  0084e8a0    00000020                 : BIOS.obj (.text:ti_sysbios_knl_Queue_empty__E)
                  0084e8c0    00000020     evmc6657_pe66.oe66 (.text:ti_sysbios_knl_Swi_Module_startup__E)
                  0084e8e0    00000020     sysbios.lib : BIOS.obj (.text:ti_sysbios_knl_Swi_disable__E)
                  0084e900    00000020     evmc6657_pe66.oe66 (.text:ti_sysbios_knl_Task_Module_startup__E)
                  0084e920    00000020     evmc6657_pe66.oe66 (.text:ti_sysbios_knl_Task_SupportProxy_Module__startupDone__S)
                  0084e940    00000020     evmc6657_pe66.oe66 (.text:ti_sysbios_knl_Task_SupportProxy_checkStack__E)
                  0084e960    00000020     evmc6657_pe66.oe66 (.text:ti_sysbios_knl_Task_SupportProxy_getStackAlignment__E)
                  0084e980    00000020     evmc6657_pe66.oe66 (.text:ti_sysbios_knl_Task_SupportProxy_start__E)
                  0084e9a0    00000020     evmc6657_pe66.oe66 (.text:ti_sysbios_knl_Task_SupportProxy_swap__E)
                  0084e9c0    00000020     sysbios.lib : BIOS.obj (.text:ti_sysbios_knl_Task_disable__E)
                  0084e9e0    00000020     evmc6657_pe66.oe66 (.text:ti_sysbios_timers_timer64_Timer_Module__startupDone__S)
                  0084ea00    00000020     evmc6657_pe66.oe66 (.text:ti_sysbios_timers_timer64_Timer_Module_startup__E)
                  0084ea20    00000020     evmc6657_pe66.oe66 (.text:ti_sysbios_timers_timer64_Timer_TimerSupportProxy_enable__E)
                  0084ea40    00000020     sysbios.lib : BIOS.obj (.text:ti_sysbios_timers_timer64_Timer_setNextTick__E)
                  0084ea60    00000020     evmc6657_pe66.oe66 (.text:xdc_iargToPtr)
                  0084ea80    00000020     evmc6657_pe66.oe66 (.text:xdc_runtime_Error_check__E)
                  0084eaa0    00000020     evmc6657_pe66.oe66 (.text:xdc_runtime_Error_init__E)
                  0084eac0    00000020     evmc6657_pe66.oe66 (.text:xdc_runtime_Error_print__E)
                  0084eae0    00000020     evmc6657_pe66.oe66 (.text:xdc_runtime_Gate_enterSystem__E)
                  0084eb00    00000020     ti.targets.rts6000.ae66 : Gate.oe66 (.text:xdc_runtime_Gate_enterSystem__F)
                  0084eb20    00000020     evmc6657_pe66.oe66 (.text:xdc_runtime_Gate_leaveSystem__E)
                  0084eb40    00000020     evmc6657_pe66.oe66 (.text:xdc_runtime_Memory_HeapProxy_alloc__E)
                  0084eb60    00000020     evmc6657_pe66.oe66 (.text:xdc_runtime_Memory_HeapProxy_free__E)
                  0084eb80    00000020     evmc6657_pe66.oe66 (.text:xdc_runtime_Memory_alloc__E)
                  0084eba0    00000020     evmc6657_pe66.oe66 (.text:xdc_runtime_Memory_calloc__E)
                  0084ebc0    00000020     evmc6657_pe66.oe66 (.text:xdc_runtime_Memory_free__E)
                  0084ebe0    00000020     evmc6657_pe66.oe66 (.text:xdc_runtime_Registry_findById__E)
                  0084ec00    00000020     evmc6657_pe66.oe66 (.text:xdc_runtime_Startup_exec__E)
                  0084ec20    00000020     evmc6657_pe66.oe66 (.text:xdc_runtime_Startup_reset__I)
                  0084ec40    00000020     evmc6657_pe66.oe66 (.text:xdc_runtime_SysStd_abort__E)
                  0084ec60    00000020     evmc6657_pe66.oe66 (.text:xdc_runtime_SysStd_exit__E)
                  0084ec80    00000020     ti.targets.rts6000.ae66 : SysStd.oe66 (.text:xdc_runtime_SysStd_exit__F)
                  0084eca0    00000020     evmc6657_pe66.oe66 (.text:xdc_runtime_SysStd_putch__E)
                  0084ecc0    00000020     ti.targets.rts6000.ae66 : SysStd.oe66 (.text:xdc_runtime_SysStd_putch__F)
                  0084ece0    00000020     evmc6657_pe66.oe66 (.text:xdc_runtime_SysStd_ready__E)
                  0084ed00    00000020     ti.targets.rts6000.ae66 : SysStd.oe66 (.text:xdc_runtime_SysStd_ready__F)
                  0084ed20    00000020     evmc6657_pe66.oe66 (.text:xdc_runtime_System_Module_GateProxy_enter__E)
                  0084ed40    00000020     evmc6657_pe66.oe66 (.text:xdc_runtime_System_Module_GateProxy_leave__E)
                  0084ed60    00000020     evmc6657_pe66.oe66 (.text:xdc_runtime_System_Module_startup__E)
                  0084ed80    00000020     ti.targets.rts6000.ae66 : System.oe66 (.text:xdc_runtime_System_Module_startup__F)
                  0084eda0    00000020     evmc6657_pe66.oe66 (.text:xdc_runtime_System_SupportProxy_abort__E)
                  0084edc0    00000020     evmc6657_pe66.oe66 (.text:xdc_runtime_System_SupportProxy_exit__E)
                  0084ede0    00000020     evmc6657_pe66.oe66 (.text:xdc_runtime_System_SupportProxy_putch__E)
                  0084ee00    00000020     evmc6657_pe66.oe66 (.text:xdc_runtime_System_SupportProxy_ready__E)
                  0084ee20    00000020     evmc6657_pe66.oe66 (.text:xdc_runtime_System_abort__E)
                  0084ee40    00000020     evmc6657_pe66.oe66 (.text:xdc_runtime_System_atexit__E)
                  0084ee60    00000020     evmc6657_pe66.oe66 (.text:xdc_runtime_System_exit__E)
                  0084ee80    00000020     ti.targets.rts6000.ae66 : System.oe66 (.text:xdc_runtime_System_exit__F)
                  0084eea0    00000020                             : System.oe66 (.text:xdc_runtime_System_lastFxn__I)
                  0084eec0    00000020     evmc6657_pe66.oe66 (.text:xdc_runtime_System_vsprintf__E)
                  0084eee0    00000020     ti.targets.rts6000.ae66 : System.oe66 (.text:xdc_runtime_System_vsprintf__F)
                  0084ef00    00000020     evmc6657_pe66.oe66 (.text:xdc_runtime_Text_cordText__E)
                  0084ef20    00000020     evmc6657_pe66.oe66 (.text:xdc_runtime_Text_putLab__E)
                  0084ef40    00000020     evmc6657_pe66.oe66 (.text:xdc_runtime_Text_putSite__E)
                  0084ef60    00000020     evmc6657_pe66.oe66 (.text:xdc_runtime_Text_ropeText__E)

systemHeapMaster 
*          0    0084ef80    00008000     UNINITIALIZED
                  0084ef80    00008000     evmc6657_pe66.oe66 (systemHeapMaster)

.const     0    00856f80    00003102     
                  00856f80    000011d6     evmc6657_pe66.oe66 (.const:xdc_runtime_Text_charTab__A)
                  00858156    00000840     ti.drv.emac.ae66 : emac_drv.oe66 (.const:.string)
                  00858996    00000002     --HOLE-- [fill = 0]
                  00858998    00000464     my_test_main.obj (.const:.string)
                  00858dfc    0000042c     sysbios.lib : BIOS.obj (.const:.string)
                  00859228    00000400     evmc6657_pe66.oe66 (.const:ti_sysbios_family_c66_Cache_marvalues__C)
                  00859628    00000101     rts6600_elf.lib : ctype.obj (.const:.string:_ctypes_)
                  00859729    00000003     --HOLE-- [fill = 0]
                  0085972c    00000004     ti.targets.rts6000.ae66 : Assert.oe66 (.const:.string)
                  00859730    000000c8     evmc6657_pe66.oe66 (.const:xdc_runtime_Text_nodeTab__A)
                  008597f8    00000058     ti.platform.evm6657l.ae66 : platform.obj (.const:.string)
                  00859850    00000058     ti.targets.rts6000.ae66 : Error.oe66 (.const:.string)
                  008598a8    00000054     evmc6657_pe66.oe66 (.const:.string)
                  008598fc    00000040     ti.targets.rts6000.ae66 : Text.oe66 (.const:.string)
                  0085993c    00000038     evmc6657_pe66.oe66 (.const:ti_sysbios_knl_Task_Object__PARAMS__C)
                  00859974    00000030     evmc6657_pe66.oe66 (.const:ti_sysbios_family_c64p_Hwi_Object__PARAMS__C)
                  008599a4    00000004     evmc6657_pe66.oe66 (.const:ti_sysbios_BIOS_Module__diagsEnabled__C)
                  008599a8    0000002f     ti.drv.emac.ae66 : emac_drv.oe66 (.const:.string:emac_version_str)
                  008599d7    00000001     --HOLE-- [fill = 0]
                  008599d8    0000002c     ti.targets.rts6000.ae66 : Startup.oe66 (.const:.string)
                  00859a04    0000002c     evmc6657_pe66.oe66 (.const:ti_sysbios_hal_Hwi_Object__PARAMS__C)
                  00859a30    00000028     ti.platform.evm6657l.ae66 : evmc665x_nand.obj (.const:.string:$P$T0$1)
                  00859a58    00000028                               : evmc665x_nand.obj (.const:.string:$P$T1$2)
                  00859a80    00000028     evmc6657_pe66.oe66 (.const:ti_sysbios_heaps_HeapMem_Module__FXNS__C)
                  00859aa8    00000028     evmc6657_pe66.oe66 (.const:xdc_runtime_Startup_sfxnTab__A)
                  00859ad0    00000024     evmc6657_pe66.oe66 (.const:ti_sysbios_gates_GateHwi_Module__FXNS__C)
                  00859af4    00000024     evmc6657_pe66.oe66 (.const:ti_sysbios_gates_GateMutex_Module__FXNS__C)
                  00859b18    00000024     evmc6657_pe66.oe66 (.const:ti_sysbios_knl_Clock_Object__PARAMS__C)
                  00859b3c    00000024     evmc6657_pe66.oe66 (.const:ti_sysbios_knl_Semaphore_Object__PARAMS__C)
                  00859b60    00000023     rts6600_elf.lib : _printfi.obj (.const:.string)
                  00859b83    00000001     --HOLE-- [fill = 0]
                  00859b84    00000020     ti.targets.rts6000.ae66 : Core-mem.oe66 (.const:.string)
                  00859ba4    00000020     evmc6657_pe66.oe66 (.const:ti_sysbios_family_c64p_Hwi_Object__DESC__C)
                  00859bc4    00000020     evmc6657_pe66.oe66 (.const:ti_sysbios_gates_GateHwi_Object__DESC__C)
                  00859be4    00000020     evmc6657_pe66.oe66 (.const:ti_sysbios_gates_GateMutex_Object__DESC__C)
                  00859c04    00000020     evmc6657_pe66.oe66 (.const:ti_sysbios_hal_Hwi_Object__DESC__C)
                  00859c24    00000020     evmc6657_pe66.oe66 (.const:ti_sysbios_heaps_HeapMem_Object__DESC__C)
                  00859c44    00000020     evmc6657_pe66.oe66 (.const:ti_sysbios_heaps_HeapMem_Object__PARAMS__C)
                  00859c64    00000020     evmc6657_pe66.oe66 (.const:ti_sysbios_knl_Clock_Object__DESC__C)
                  00859c84    00000020     evmc6657_pe66.oe66 (.const:ti_sysbios_knl_Queue_Object__DESC__C)
                  00859ca4    00000020     evmc6657_pe66.oe66 (.const:ti_sysbios_knl_Semaphore_Object__DESC__C)
                  00859cc4    00000020     evmc6657_pe66.oe66 (.const:ti_sysbios_knl_Task_Object__DESC__C)
                  00859ce4    00000004     evmc6657_pe66.oe66 (.const:ti_sysbios_BIOS_Module__diagsIncluded__C)
                  00859ce8    00000018     my_test_main.obj (.const:$P$T0$1)
                  00859d00    00000018     evmc6657_pe66.oe66 (.const:ti_sysbios_gates_GateHwi_Object__PARAMS__C)
                  00859d18    00000018     evmc6657_pe66.oe66 (.const:ti_sysbios_gates_GateMutex_Object__PARAMS__C)
                  00859d30    00000018     evmc6657_pe66.oe66 (.const:ti_sysbios_knl_Queue_Object__PARAMS__C)
                  00859d48    00000018     evmc6657_pe66.oe66 (.const:ti_sysbios_knl_Task_hooks__A)
                  00859d60    00000014     evmc6657_pe66.oe66 (.const:xdc_runtime_Startup_sfxnRts__A)
                  00859d74    0000000c     evmc6657_pe66.oe66 (.const:ti_sysbios_family_c66_Cache_initSize__C)
                  00859d80    00000011     ti.targets.rts6000.ae66 : System.oe66 (.const:digtohex)
                  00859d91    00000003     --HOLE-- [fill = 0]
                  00859d94    00000004     evmc6657_pe66.oe66 (.const:ti_sysbios_BIOS_Module__diagsMask__C)
                  00859d98    0000000c     evmc6657_pe66.oe66 (.const:xdc_runtime_Startup_firstFxns__A)
                  00859da4    00000008     ti.targets.rts6000.ae66 : System.oe66 (.const:.string)
                  00859dac    00000008     evmc6657_pe66.oe66 (.const:ti_sysbios_knl_Idle_funcList__C)
                  00859db4    00000008     evmc6657_pe66.oe66 (.const:ti_sysbios_knl_Task_hooks__C)
                  00859dbc    00000008     evmc6657_pe66.oe66 (.const:xdc_runtime_Startup_firstFxns__C)
                  00859dc4    00000008     evmc6657_pe66.oe66 (.const:xdc_runtime_Startup_lastFxns__C)
                  00859dcc    00000004     evmc6657_pe66.oe66 (.const:ti_sysbios_BIOS_installedErrorHook__C)
                  00859dd0    00000006     my_test_main.obj (.const:.string:$P$T1$2)
                  00859dd6    00000002     --HOLE-- [fill = 0]
                  00859dd8    00000004     evmc6657_pe66.oe66 (.const:ti_sysbios_family_c62_TaskSupport_stackAlignment__C)
                  00859ddc    00000004     evmc6657_pe66.oe66 (.const:ti_sysbios_family_c64p_Exception_E_exceptionMin__C)
                  00859de0    00000004     evmc6657_pe66.oe66 (.const:ti_sysbios_family_c64p_Exception_exceptionHook__C)
                  00859de4    00000004     evmc6657_pe66.oe66 (.const:ti_sysbios_family_c64p_Exception_externalHook__C)
                  00859de8    00000004     evmc6657_pe66.oe66 (.const:ti_sysbios_family_c64p_Exception_internalHook__C)
                  00859dec    00000004     evmc6657_pe66.oe66 (.const:ti_sysbios_family_c64p_Exception_nmiHook__C)
                  00859df0    00000004     evmc6657_pe66.oe66 (.const:ti_sysbios_family_c64p_Hwi_E_alreadyDefined__C)
                  00859df4    00000004     evmc6657_pe66.oe66 (.const:ti_sysbios_family_c64p_Hwi_E_handleNotFound__C)
                  00859df8    00000004     evmc6657_pe66.oe66 (.const:ti_sysbios_family_c64p_Hwi_LD_end__C)
                  00859dfc    00000004     evmc6657_pe66.oe66 (.const:ti_sysbios_family_c64p_Hwi_LM_begin__C)
                  00859e00    00000004     evmc6657_pe66.oe66 (.const:ti_sysbios_family_c64p_Hwi_Module__diagsEnabled__C)
                  00859e04    00000004     evmc6657_pe66.oe66 (.const:ti_sysbios_family_c64p_Hwi_Module__diagsIncluded__C)
                  00859e08    00000004     evmc6657_pe66.oe66 (.const:ti_sysbios_family_c64p_Hwi_Module__diagsMask__C)
                  00859e0c    00000004     evmc6657_pe66.oe66 (.const:ti_sysbios_family_c64p_Hwi_Module__loggerFxn1__C)
                  00859e10    00000004     evmc6657_pe66.oe66 (.const:ti_sysbios_family_c64p_Hwi_Module__loggerFxn8__C)
                  00859e14    00000004     evmc6657_pe66.oe66 (.const:ti_sysbios_family_c64p_Hwi_Module__loggerObj__C)
                  00859e18    00000004     evmc6657_pe66.oe66 (.const:ti_sysbios_family_c66_Cache_atomicBlockSize__C)
                  00859e1c    00000004     evmc6657_pe66.oe66 (.const:ti_sysbios_gates_GateMutex_A_badContext__C)
                  00859e20    00000004     evmc6657_pe66.oe66 (.const:ti_sysbios_gates_GateMutex_Instance_State_sem__O)
                  00859e24    00000004     evmc6657_pe66.oe66 (.const:ti_sysbios_gates_GateMutex_Module__diagsEnabled__C)
                  00859e28    00000004     evmc6657_pe66.oe66 (.const:ti_sysbios_gates_GateMutex_Module__diagsIncluded__C)
                  00859e2c    00000004     evmc6657_pe66.oe66 (.const:ti_sysbios_gates_GateMutex_Module__diagsMask__C)
                  00859e30    00000004     evmc6657_pe66.oe66 (.const:ti_sysbios_hal_Hwi_E_stackOverflow__C)
                  00859e34    00000004     evmc6657_pe66.oe66 (.const:ti_sysbios_heaps_HeapMem_A_align__C)
                  00859e38    00000004     evmc6657_pe66.oe66 (.const:ti_sysbios_heaps_HeapMem_A_heapSize__C)
                  00859e3c    00000004     evmc6657_pe66.oe66 (.const:ti_sysbios_heaps_HeapMem_A_invalidFree__C)
                  00859e40    00000004     evmc6657_pe66.oe66 (.const:ti_sysbios_heaps_HeapMem_A_zeroBlock__C)
                  00859e44    00000004     evmc6657_pe66.oe66 (.const:ti_sysbios_heaps_HeapMem_E_memory__C)
                  00859e48    00000004     evmc6657_pe66.oe66 (.const:ti_sysbios_heaps_HeapMem_Module__diagsEnabled__C)
                  00859e4c    00000004     evmc6657_pe66.oe66 (.const:ti_sysbios_heaps_HeapMem_Module__diagsIncluded__C)
                  00859e50    00000004     evmc6657_pe66.oe66 (.const:ti_sysbios_heaps_HeapMem_Module__diagsMask__C)
                  00859e54    00000004     evmc6657_pe66.oe66 (.const:ti_sysbios_heaps_HeapMem_Module__gateObj__C)
                  00859e58    00000004     evmc6657_pe66.oe66 (.const:ti_sysbios_heaps_HeapMem_Object__count__C)
                  00859e5c    00000004     evmc6657_pe66.oe66 (.const:ti_sysbios_heaps_HeapMem_Object__table__C)
                  00859e60    00000004     evmc6657_pe66.oe66 (.const:ti_sysbios_heaps_HeapMem_reqAlignMask__C)
                  00859e64    00000004     evmc6657_pe66.oe66 (.const:ti_sysbios_heaps_HeapMem_reqAlign__C)
                  00859e68    00000004     evmc6657_pe66.oe66 (.const:ti_sysbios_knl_Clock_A_badThreadType__C)
                  00859e6c    00000004     evmc6657_pe66.oe66 (.const:ti_sysbios_knl_Clock_LM_begin__C)
                  00859e70    00000004     evmc6657_pe66.oe66 (.const:ti_sysbios_knl_Clock_LM_tick__C)
                  00859e74    00000004     evmc6657_pe66.oe66 (.const:ti_sysbios_knl_Clock_LW_delayed__C)
                  00859e78    00000004     evmc6657_pe66.oe66 (.const:ti_sysbios_knl_Clock_Module_State_clockQ__O)
                  00859e7c    00000004     evmc6657_pe66.oe66 (.const:ti_sysbios_knl_Clock_Module__diagsEnabled__C)
                  00859e80    00000004     evmc6657_pe66.oe66 (.const:ti_sysbios_knl_Clock_Module__diagsIncluded__C)
                  00859e84    00000004     evmc6657_pe66.oe66 (.const:ti_sysbios_knl_Clock_Module__diagsMask__C)
                  00859e88    00000004     evmc6657_pe66.oe66 (.const:ti_sysbios_knl_Clock_Module__loggerFxn1__C)
                  00859e8c    00000004     evmc6657_pe66.oe66 (.const:ti_sysbios_knl_Clock_Module__loggerFxn2__C)
                  00859e90    00000004     evmc6657_pe66.oe66 (.const:ti_sysbios_knl_Clock_Module__loggerObj__C)
                  00859e94    00000004     evmc6657_pe66.oe66 (.const:ti_sysbios_knl_Clock_tickMode__C)
                  00859e98    00000004     evmc6657_pe66.oe66 (.const:ti_sysbios_knl_Clock_tickSource__C)
                  00859e9c    00000004     evmc6657_pe66.oe66 (.const:ti_sysbios_knl_Queue_Object__count__C)
                  00859ea0    00000004     evmc6657_pe66.oe66 (.const:ti_sysbios_knl_Idle_funcList__A)
                  00859ea4    00000004     evmc6657_pe66.oe66 (.const:ti_sysbios_knl_Queue_Object__table__C)
                  00859ea8    00000004     evmc6657_pe66.oe66 (.const:ti_sysbios_knl_Semaphore_A_badContext__C)
                  00859eac    00000004     evmc6657_pe66.oe66 (.const:ti_sysbios_knl_Semaphore_A_noEvents__C)
                  00859eb0    00000004     evmc6657_pe66.oe66 (.const:ti_sysbios_knl_Semaphore_A_overflow__C)
                  00859eb4    00000004     evmc6657_pe66.oe66 (.const:ti_sysbios_knl_Semaphore_Instance_State_pendQ__O)
                  00859eb8    00000004     evmc6657_pe66.oe66 (.const:ti_sysbios_knl_Semaphore_LM_pend__C)
                  00859ebc    00000004     evmc6657_pe66.oe66 (.const:ti_sysbios_knl_Semaphore_LM_post__C)
                  00859ec0    00000004     evmc6657_pe66.oe66 (.const:ti_sysbios_knl_Semaphore_Module__diagsEnabled__C)
                  00859ec4    00000004     evmc6657_pe66.oe66 (.const:ti_sysbios_knl_Semaphore_Module__diagsIncluded__C)
                  00859ec8    00000004     evmc6657_pe66.oe66 (.const:ti_sysbios_knl_Semaphore_Module__diagsMask__C)
                  00859ecc    00000004     evmc6657_pe66.oe66 (.const:ti_sysbios_knl_Semaphore_Module__loggerFxn2__C)
                  00859ed0    00000004     evmc6657_pe66.oe66 (.const:ti_sysbios_knl_Semaphore_Module__loggerFxn4__C)
                  00859ed4    00000004     evmc6657_pe66.oe66 (.const:ti_sysbios_knl_Semaphore_Module__loggerObj__C)
                  00859ed8    00000004     evmc6657_pe66.oe66 (.const:ti_sysbios_knl_Swi_LD_end__C)
                  00859edc    00000004     evmc6657_pe66.oe66 (.const:ti_sysbios_knl_Swi_LM_begin__C)
                  00859ee0    00000004     evmc6657_pe66.oe66 (.const:ti_sysbios_knl_Swi_LM_post__C)
                  00859ee4    00000004     evmc6657_pe66.oe66 (.const:ti_sysbios_knl_Swi_Module__diagsEnabled__C)
                  00859ee8    00000004     evmc6657_pe66.oe66 (.const:ti_sysbios_knl_Swi_Module__diagsIncluded__C)
                  00859eec    00000004     evmc6657_pe66.oe66 (.const:ti_sysbios_knl_Swi_Module__diagsMask__C)
                  00859ef0    00000004     evmc6657_pe66.oe66 (.const:ti_sysbios_knl_Swi_Module__loggerFxn1__C)
                  00859ef4    00000004     evmc6657_pe66.oe66 (.const:ti_sysbios_knl_Swi_Module__loggerFxn4__C)
                  00859ef8    00000004     evmc6657_pe66.oe66 (.const:ti_sysbios_knl_Swi_Module__loggerObj__C)
                  00859efc    00000004     evmc6657_pe66.oe66 (.const:ti_sysbios_knl_Swi_Object__count__C)
                  00859f00    00000004     evmc6657_pe66.oe66 (.const:ti_sysbios_knl_Swi_Object__table__C)
                  00859f04    00000004     evmc6657_pe66.oe66 (.const:ti_sysbios_knl_Task_A_badPriority__C)
                  00859f08    00000004     evmc6657_pe66.oe66 (.const:ti_sysbios_knl_Task_A_badTaskState__C)
                  00859f0c    00000004     evmc6657_pe66.oe66 (.const:ti_sysbios_knl_Task_A_badThreadType__C)
                  00859f10    00000004     evmc6657_pe66.oe66 (.const:ti_sysbios_knl_Task_A_noPendElem__C)
                  00859f14    00000004     evmc6657_pe66.oe66 (.const:ti_sysbios_knl_Task_E_spOutOfBounds__C)
                  00859f18    00000004     evmc6657_pe66.oe66 (.const:ti_sysbios_knl_Task_E_stackOverflow__C)
                  00859f1c    00000004     evmc6657_pe66.oe66 (.const:ti_sysbios_knl_Task_LD_block__C)
                  00859f20    00000004     evmc6657_pe66.oe66 (.const:ti_sysbios_knl_Task_LD_exit__C)
                  00859f24    00000004     evmc6657_pe66.oe66 (.const:ti_sysbios_knl_Task_LD_ready__C)
                  00859f28    00000004     evmc6657_pe66.oe66 (.const:ti_sysbios_knl_Task_LM_switch__C)
                  00859f2c    00000004     evmc6657_pe66.oe66 (.const:ti_sysbios_knl_Task_Module_State_inactiveQ__O)
                  00859f30    00000004     evmc6657_pe66.oe66 (.const:ti_sysbios_knl_Task_Module_State_terminatedQ__O)
                  00859f34    00000004     evmc6657_pe66.oe66 (.const:ti_sysbios_knl_Task_Module__diagsEnabled__C)
                  00859f38    00000004     evmc6657_pe66.oe66 (.const:ti_sysbios_knl_Task_Module__diagsIncluded__C)
                  00859f3c    00000004     evmc6657_pe66.oe66 (.const:ti_sysbios_knl_Task_Module__diagsMask__C)
                  00859f40    00000004     evmc6657_pe66.oe66 (.const:ti_sysbios_knl_Task_Module__loggerFxn2__C)
                  00859f44    00000004     evmc6657_pe66.oe66 (.const:ti_sysbios_knl_Task_Module__loggerFxn4__C)
                  00859f48    00000004     evmc6657_pe66.oe66 (.const:ti_sysbios_knl_Task_Module__loggerObj__C)
                  00859f4c    00000004     evmc6657_pe66.oe66 (.const:ti_sysbios_knl_Task_Object__count__C)
                  00859f50    00000004     evmc6657_pe66.oe66 (.const:ti_sysbios_knl_Task_Object__heap__C)
                  00859f54    00000004     evmc6657_pe66.oe66 (.const:ti_sysbios_knl_Task_Object__table__C)
                  00859f58    00000004     evmc6657_pe66.oe66 (.const:ti_sysbios_knl_Task_allBlockedFunc__C)
                  00859f5c    00000004     evmc6657_pe66.oe66 (.const:ti_sysbios_knl_Task_defaultStackHeap__C)
                  00859f60    00000004     evmc6657_pe66.oe66 (.const:ti_sysbios_knl_Task_defaultStackSize__C)
                  00859f64    00000004     evmc6657_pe66.oe66 (.const:ti_sysbios_knl_Task_numConstructedTasks__C)
                  00859f68    00000004     evmc6657_pe66.oe66 (.const:ti_sysbios_knl_Task_numPriorities__C)
                  00859f6c    00000004     evmc6657_pe66.oe66 (.const:ti_sysbios_timers_timer64_Timer_A_notAvailable__C)
                  00859f70    00000004     evmc6657_pe66.oe66 (.const:ti_sysbios_timers_timer64_Timer_E_cannotSupport__C)
                  00859f74    00000004     evmc6657_pe66.oe66 (.const:ti_sysbios_timers_timer64_Timer_Module__diagsEnabled__C)
                  00859f78    00000004     evmc6657_pe66.oe66 (.const:ti_sysbios_timers_timer64_Timer_Module__diagsIncluded__C)
                  00859f7c    00000004     evmc6657_pe66.oe66 (.const:ti_sysbios_timers_timer64_Timer_Module__diagsMask__C)
                  00859f80    00000004     evmc6657_pe66.oe66 (.const:ti_sysbios_timers_timer64_Timer_anyMask__C)
                  00859f84    00000004     evmc6657_pe66.oe66 (.const:ti_sysbios_timers_timer64_Timer_freqDivisor__C)
                  00859f88    00000004     evmc6657_pe66.oe66 (.const:ti_sysbios_timers_timer64_Timer_numLocalTimers__C)
                  00859f8c    00000004     evmc6657_pe66.oe66 (.const:ti_sysbios_timers_timer64_Timer_numTimerDevices__C)
                  00859f90    00000004     evmc6657_pe66.oe66 (.const:xdc_runtime_Assert_E_assertFailed__C)
                  00859f94    00000004     evmc6657_pe66.oe66 (.const:xdc_runtime_Core_A_initializedParams__C)
                  00859f98    00000004     evmc6657_pe66.oe66 (.const:xdc_runtime_Core_Module__diagsEnabled__C)
                  00859f9c    00000004     evmc6657_pe66.oe66 (.const:xdc_runtime_Core_Module__diagsIncluded__C)
                  00859fa0    00000004     evmc6657_pe66.oe66 (.const:xdc_runtime_Core_Module__diagsMask__C)
                  00859fa4    00000004     evmc6657_pe66.oe66 (.const:xdc_runtime_Error_E_generic__C)
                  00859fa8    00000004     evmc6657_pe66.oe66 (.const:xdc_runtime_Error_E_memory__C)
                  00859fac    00000004     evmc6657_pe66.oe66 (.const:xdc_runtime_Error_Module__diagsEnabled__C)
                  00859fb0    00000004     evmc6657_pe66.oe66 (.const:xdc_runtime_Error_Module__diagsIncluded__C)
                  00859fb4    00000004     evmc6657_pe66.oe66 (.const:xdc_runtime_Error_Module__diagsMask__C)
                  00859fb8    00000004     evmc6657_pe66.oe66 (.const:xdc_runtime_Error_Module__loggerFxn8__C)
                  00859fbc    00000004     evmc6657_pe66.oe66 (.const:xdc_runtime_Error_Module__loggerObj__C)
                  00859fc0    00000004     evmc6657_pe66.oe66 (.const:xdc_runtime_Error_policy__C)
                  00859fc4    00000004     evmc6657_pe66.oe66 (.const:xdc_runtime_Error_raiseHook__C)
                  00859fc8    00000004     evmc6657_pe66.oe66 (.const:xdc_runtime_IGateProvider_Interface__BASE__C)
                  00859fcc    00000004     evmc6657_pe66.oe66 (.const:xdc_runtime_IHeap_Interface__BASE__C)
                  00859fd0    00000004     evmc6657_pe66.oe66 (.const:xdc_runtime_IModule_Interface__BASE__C)
                  00859fd4    00000004     evmc6657_pe66.oe66 (.const:xdc_runtime_Log_L_error__C)
                  00859fd8    00000004     evmc6657_pe66.oe66 (.const:xdc_runtime_Memory_defaultHeapInstance__C)
                  00859fdc    00000004     evmc6657_pe66.oe66 (.const:xdc_runtime_Startup_execImpl__C)
                  00859fe0    00000004     evmc6657_pe66.oe66 (.const:xdc_runtime_Startup_lastFxns__A)
                  00859fe4    00000004     evmc6657_pe66.oe66 (.const:xdc_runtime_Startup_maxPasses__C)
                  00859fe8    00000004     evmc6657_pe66.oe66 (.const:xdc_runtime_Startup_sfxnRts__C)
                  00859fec    00000004     evmc6657_pe66.oe66 (.const:xdc_runtime_Startup_sfxnTab__C)
                  00859ff0    00000004     evmc6657_pe66.oe66 (.const:xdc_runtime_Startup_startModsFxn__C)
                  00859ff4    00000004     evmc6657_pe66.oe66 (.const:xdc_runtime_System_Module__gateObj__C)
                  00859ff8    00000004     evmc6657_pe66.oe66 (.const:xdc_runtime_System_extendFxn__C)
                  00859ffc    00000004     evmc6657_pe66.oe66 (.const:xdc_runtime_System_maxAtexitHandlers__C)
                  0085a000    00000004     evmc6657_pe66.oe66 (.const:xdc_runtime_Text_charTab__C)
                  0085a004    00000004     evmc6657_pe66.oe66 (.const:xdc_runtime_Text_nameEmpty__C)
                  0085a008    00000004     evmc6657_pe66.oe66 (.const:xdc_runtime_Text_nameStatic__C)
                  0085a00c    00000004     evmc6657_pe66.oe66 (.const:xdc_runtime_Text_nameUnknown__C)
                  0085a010    00000004     evmc6657_pe66.oe66 (.const:xdc_runtime_Text_nodeTab__C)
                  0085a014    00000004     evmc6657_pe66.oe66 (.const:xdc_runtime_Text_visitRopeFxn__C)
                  0085a018    00000002     evmc6657_pe66.oe66 (.const:ti_sysbios_BIOS_Module__id__C)
                  0085a01a    00000002     --HOLE-- [fill = 0]
                  0085a01c    00000002     evmc6657_pe66.oe66 (.const:ti_sysbios_family_c64p_Exception_Module__id__C)
                  0085a01e    00000002     --HOLE-- [fill = 0]
                  0085a020    00000002     evmc6657_pe66.oe66 (.const:ti_sysbios_family_c64p_Hwi_Module__id__C)
                  0085a022    00000002     --HOLE-- [fill = 0]
                  0085a024    00000002     evmc6657_pe66.oe66 (.const:ti_sysbios_family_c64p_Hwi_Module__loggerDefined__C)
                  0085a026    00000002     --HOLE-- [fill = 0]
                  0085a028    00000002     evmc6657_pe66.oe66 (.const:ti_sysbios_gates_GateMutex_Module__id__C)
                  0085a02a    00000002     --HOLE-- [fill = 0]
                  0085a02c    00000002     evmc6657_pe66.oe66 (.const:ti_sysbios_hal_Hwi_Module__id__C)
                  0085a02e    00000002     --HOLE-- [fill = 0]
                  0085a030    00000002     evmc6657_pe66.oe66 (.const:ti_sysbios_heaps_HeapMem_Module__id__C)
                  0085a032    00000002     --HOLE-- [fill = 0]
                  0085a034    00000002     evmc6657_pe66.oe66 (.const:ti_sysbios_knl_Clock_Module__id__C)
                  0085a036    00000002     --HOLE-- [fill = 0]
                  0085a038    00000002     evmc6657_pe66.oe66 (.const:ti_sysbios_knl_Clock_Module__loggerDefined__C)
                  0085a03a    00000002     --HOLE-- [fill = 0]
                  0085a03c    00000002     evmc6657_pe66.oe66 (.const:ti_sysbios_knl_Semaphore_Module__id__C)
                  0085a03e    00000002     --HOLE-- [fill = 0]
                  0085a040    00000002     evmc6657_pe66.oe66 (.const:ti_sysbios_knl_Semaphore_Module__loggerDefined__C)
                  0085a042    00000002     --HOLE-- [fill = 0]
                  0085a044    00000002     evmc6657_pe66.oe66 (.const:ti_sysbios_knl_Swi_Module__id__C)
                  0085a046    00000002     --HOLE-- [fill = 0]
                  0085a048    00000002     evmc6657_pe66.oe66 (.const:ti_sysbios_knl_Swi_Module__loggerDefined__C)
                  0085a04a    00000002     --HOLE-- [fill = 0]
                  0085a04c    00000002     evmc6657_pe66.oe66 (.const:ti_sysbios_knl_Task_Module__id__C)
                  0085a04e    00000002     --HOLE-- [fill = 0]
                  0085a050    00000002     evmc6657_pe66.oe66 (.const:ti_sysbios_knl_Task_Module__loggerDefined__C)
                  0085a052    00000002     --HOLE-- [fill = 0]
                  0085a054    00000002     evmc6657_pe66.oe66 (.const:ti_sysbios_knl_Task_deleteTerminatedTasks__C)
                  0085a056    00000002     --HOLE-- [fill = 0]
                  0085a058    00000002     evmc6657_pe66.oe66 (.const:ti_sysbios_knl_Task_initStackFlag__C)
                  0085a05a    00000002     --HOLE-- [fill = 0]
                  0085a05c    00000002     evmc6657_pe66.oe66 (.const:ti_sysbios_timers_timer64_Timer_Module__id__C)
                  0085a05e    00000002     --HOLE-- [fill = 0]
                  0085a060    00000002     evmc6657_pe66.oe66 (.const:ti_sysbios_timers_timer64_Timer_startupNeeded__C)
                  0085a062    00000002     --HOLE-- [fill = 0]
                  0085a064    00000002     evmc6657_pe66.oe66 (.const:xdc_runtime_Core_Module__id__C)
                  0085a066    00000002     --HOLE-- [fill = 0]
                  0085a068    00000002     evmc6657_pe66.oe66 (.const:xdc_runtime_Error_Module__loggerDefined__C)
                  0085a06a    00000002     --HOLE-- [fill = 0]
                  0085a06c    00000002     evmc6657_pe66.oe66 (.const:xdc_runtime_Error_maxDepth__C)
                  0085a06e    00000002     --HOLE-- [fill = 0]
                  0085a070    00000002     evmc6657_pe66.oe66 (.const:xdc_runtime_Memory_Module__id__C)
                  0085a072    00000002     --HOLE-- [fill = 0]
                  0085a074    00000002     evmc6657_pe66.oe66 (.const:xdc_runtime_Text_charCnt__C)
                  0085a076    00000002     --HOLE-- [fill = 0]
                  0085a078    00000002     evmc6657_pe66.oe66 (.const:xdc_runtime_Text_isLoaded__C)
                  0085a07a    00000002     --HOLE-- [fill = 0]
                  0085a07c    00000002     evmc6657_pe66.oe66 (.const:xdc_runtime_Text_registryModsLastId__C)
                  0085a07e    00000002     --HOLE-- [fill = 0]
                  0085a080    00000002     evmc6657_pe66.oe66 (.const:xdc_runtime_Text_unnamedModsLastId__C)

.far       0    0085a088    000032d4     UNINITIALIZED
                  0085a088    00001a04     ti.drv.emac.ae66 : emac_drv.oe66 (.far:EMAC_DRV)
                  0085ba8c    0000173c     my_test_main.obj (.far:APP_EMAC)
                  0085d1c8    00000140     rts6600_elf.lib : defs.obj (.far)
                  0085d308    00000044     ti.platform.evm6657l.ae66 : evmc665x_i2c_eeprom.obj (.far)
                  0085d34c    00000004     --HOLE--
                  0085d350    00000008     rts6600_elf.lib : trgdrv.obj (.far)
                  0085d358    00000004     evmc6657_pe66.oe66 (.far)

.stack     0    0085d360    00001000     UNINITIALIZED
                  0085d360    00000008     boot.ae66 : boot.oe66 (.stack)
                  0085d368    00000ff8     --HOLE--

.fardata   0    0085e360    000008fc     
                  0085e360    000001e0     rts6600_elf.lib : defs.obj (.fardata:_ftable)
                  0085e540    000001d0     evmc6657_pe66.oe66 (.fardata)
                  0085e710    000000c0     evmc6657_pe66.oe66 (.fardata:ti_sysbios_timers_timer64_Timer_Module_State_0_device__A)
                  0085e7d0    000000a0     rts6600_elf.lib : lowlev.obj (.fardata:_stream)
                  0085e870    00000080     evmc6657_pe66.oe66 (.fardata:ti_sysbios_knl_Swi_Module_State_0_readyQ__A)
                  0085e8f0    00000080     evmc6657_pe66.oe66 (.fardata:ti_sysbios_knl_Task_Module_State_0_readyQ__A)
                  0085e970    00000078     rts6600_elf.lib : lowlev.obj (.fardata:_device)
                  0085e9e8    0000004c     evmc6657_pe66.oe66 (.fardata:ti_sysbios_timers_timer64_Timer_Object__table__V)
                  0085ea34    00000004     rts6600_elf.lib : defs.obj (.fardata)
                  0085ea38    00000044     evmc6657_pe66.oe66 (.fardata:ti_sysbios_knl_Task_Object__table__V)
                  0085ea7c    00000004     rts6600_elf.lib : dtor_list.obj (.fardata)
                  0085ea80    00000040     evmc6657_pe66.oe66 (.fardata:ti_sysbios_gates_GateMutex_Object__table__V)
                  0085eac0    00000040     evmc6657_pe66.oe66 (.fardata:ti_sysbios_timers_timer64_Timer_Module_State_0_gctrl__A)
                  0085eb00    00000040     evmc6657_pe66.oe66 (.fardata:ti_sysbios_timers_timer64_Timer_Module_State_0_handles__A)
                  0085eb40    00000040     evmc6657_pe66.oe66 (.fardata:ti_sysbios_timers_timer64_Timer_Module_State_0_intFreqs__A)
                  0085eb80    00000030     evmc6657_pe66.oe66 (.fardata:ti_sysbios_knl_Swi_Object__table__V)
                  0085ebb0    00000020     evmc6657_pe66.oe66 (.fardata:ti_sysbios_knl_Clock_Object__table__V)
                  0085ebd0    00000020     evmc6657_pe66.oe66 (.fardata:xdc_runtime_System_Module_State_0_atexitHandlers__A)
                  0085ebf0    00000018     ti.drv.emac.ae66 : mdio.oe66 (.fardata:PhyStateTimeout)
                  0085ec08    00000018     evmc6657_pe66.oe66 (.fardata:ti_sysbios_family_c64p_Hwi_Object__table__V)
                  0085ec20    00000014     evmc6657_pe66.oe66 (.fardata:ti_sysbios_heaps_HeapMem_Object__table__V)
                  0085ec34    0000000c     rts6600_elf.lib : exit.obj (.fardata)
                  0085ec40    00000008                     : _lock.obj (.fardata)
                  0085ec48    00000008     evmc6657_pe66.oe66 (.fardata:ti_sysbios_hal_Hwi_Object__table__V)
                  0085ec50    00000008     evmc6657_pe66.oe66 (.fardata:ti_sysbios_hal_Timer_Object__table__V)
                  0085ec58    00000004     evmc6657_pe66.oe66 (.fardata:ti_sysbios_gates_GateHwi_Object__table__V)

.far:taskStackSection 
*          0    0085ec60    00000800     UNINITIALIZED
                  0085ec60    00000800     evmc6657_pe66.oe66 (.far:taskStackSection)

.switch.1 
*          0    0085f460    00000014     
                  0085f460    00000014     ti.drv.emac.ae66 : mdio.oe66 (.switch:MDIO_timerTick)

emacComm   0    0085f480    00000194     UNINITIALIZED
                  0085f480    00000194     ti.drv.emac.ae66 : emac_drv.oe66 (emacComm)

.cio       0    0085f614    00000120     UNINITIALIZED
                  0085f614    00000120     rts6600_elf.lib : trgmsg.obj (.cio)

.switch.2 
*          0    0085f734    00000070     
                  0085f734    00000070     ti.csl.ae66 : csl_chip.oe66 (.switch:CSL_chipReadReg)

.bss       0    0085f7a4    00000008     UNINITIALIZED
                  0085f7a4    00000004     my_test_main.obj (.bss)
                  0085f7a8    00000004     ti.platform.evm6657l.ae66 : evmc665x_spi.obj (.bss)

.neardata 
*          0    0085f7ac    00000012     
                  0085f7ac    00000008     ti.platform.evm6657l.ae66 : platform.obj (.neardata)
                  0085f7b4    00000004     my_test_main.obj (.neardata)
                  0085f7b8    00000004     ti.drv.emac.ae66 : mdio.oe66 (.neardata)
                  0085f7bc    00000002                      : emac_drv.oe66 (.neardata)

.rodata    0    0085f7be    00000000     UNINITIALIZED

.vecs      0    0085f800    00000200     
                  0085f800    00000200     evmc6657_pe66.oe66 (.vecs)

.cinit     0    0085fa00    000005a4     
                  0085fa00    00000472     (.cinit..fardata.load) [load image, compression = rle]
                  0085fe72    00000002     --HOLE-- [fill = 0]
                  0085fe74    0000009b     (.cinit.platform_lib.load) [load image, compression = rle]
                  0085ff0f    00000001     --HOLE-- [fill = 0]
                  0085ff10    0000000f     (.cinit..neardata.load) [load image, compression = rle]
                  0085ff1f    00000001     --HOLE-- [fill = 0]
                  0085ff20    0000000c     (__TI_handler_table)
                  0085ff2c    00000008     (.cinit..bss.load) [load image, compression = zero_init]
                  0085ff34    00000008     (.cinit..far.load) [load image, compression = zero_init]
                  0085ff3c    00000008     (.cinit..far:PKTBUF_L2MEM.load) [load image, compression = zero_init]
                  0085ff44    00000008     (.cinit..far:taskStackSection.load) [load image, compression = zero_init]
                  0085ff4c    00000008     (.cinit.emacComm.load) [load image, compression = zero_init]
                  0085ff54    00000008     (.cinit.systemHeapMaster.load) [load image, compression = zero_init]
                  0085ff5c    00000048     (__TI_cinit_table)

platform_lib 
*          0    80000000    00000da0     
                  80000000    00000840     ti.platform.evm6657l.ae66 : evmc665x_nand.obj (platform_lib) [fill = 0]
                  80000840    00000458                               : platform.obj (platform_lib:uninit) [fill = 0]
                  80000c98    00000108                               : platform.obj (platform_lib:init)


LINKER GENERATED COPY TABLES

__TI_cinit_table @ 0085ff5c records: 9, size/record: 8, table size: 72
	.fardata: load addr=0085fa00, load size=00000472 bytes, run addr=0085e360, run size=000008fc bytes, compression=rle
	platform_lib: load addr=0085fe74, load size=0000009b bytes, run addr=80000000, run size=00000da0 bytes, compression=rle
	.neardata: load addr=0085ff10, load size=0000000f bytes, run addr=0085f7ac, run size=00000012 bytes, compression=rle
	.bss: load addr=0085ff2c, load size=00000008 bytes, run addr=0085f7a4, run size=00000008 bytes, compression=zero_init
	.far: load addr=0085ff34, load size=00000008 bytes, run addr=0085a088, run size=000032d4 bytes, compression=zero_init
	.far:PKTBUF_L2MEM: load addr=0085ff3c, load size=00000008 bytes, run addr=00800000, run size=00030000 bytes, compression=zero_init
	.far:taskStackSection: load addr=0085ff44, load size=00000008 bytes, run addr=0085ec60, run size=00000800 bytes, compression=zero_init
	emacComm: load addr=0085ff4c, load size=00000008 bytes, run addr=0085f480, run size=00000194 bytes, compression=zero_init
	systemHeapMaster: load addr=0085ff54, load size=00000008 bytes, run addr=0084ef80, run size=00008000 bytes, compression=zero_init


LINKER GENERATED HANDLER TABLE

__TI_handler_table @ 0085ff20 records: 3, size/record: 4, table size: 12
	index: 0, handler: __TI_zero_init
	index: 1, handler: __TI_decompress_rle24
	index: 2, handler: __TI_decompress_none


GLOBAL SYMBOLS: SORTED ALPHABETICALLY BY Name 

address    name
--------   ----
0084e1c0   C$$EXIT
0084cff8   C$$IO$$
0084dfa0   CSL_GPIO_open
00846e40   CSL_chipReadReg
00831e30   Convert_CoreLocal2GlobalAddr
008330d4   CorePllcGetHwSetup
00832e88   CorePllcHwSetup
00833a04   DDR2Init
008333a0   DDR3Init
00843d40   EMAC_RxServiceCheck
00844ec0   EMAC_TxServiceCheck
0083c3a0   EMAC_commonInit
0083e4a0   EMAC_coreDeInit
008376c0   EMAC_coreInit
00842e60   EMAC_sendPacket
00841c00   EMAC_setMulticast
00845de0   EMAC_setReceiveFilter
00834ce0   EVM_init
0084ab60   HOSTclose
008482e0   HOSTlseek
00848de0   HOSTopen
00849f60   HOSTread
008455c0   HOSTrename
0084a020   HOSTunlink
0084a0e0   HOSTwrite
0084dfc0   MDIO_getStatus
0084e000   MDIO_initPHY
0084b600   MDIO_open
00838620   MDIO_timerTick
00835e78   NandGetDetails
008354f0   NandReadSpareArea
008358b0   NandWriteDataBytes
00835ba0   NandWriteSpareArea
0083f838   Osal_emacBeginMemAccess
0083f874   Osal_emacEndMemAccess
0083f8f8   Osal_emacEnterMultipleCoreCriticalSection
0083f8b0   Osal_emacEnterSingleCoreCriticalSection
0083f908   Osal_emacExitMultipleCoreCriticalSection
0083f8d4   Osal_emacExitSingleCoreCriticalSection
0083f948   Osal_emacFree
0083f918   Osal_emacMalloc
0083f7e8   Osal_platformFree
0083f7b4   Osal_platformMalloc
0083f810   Osal_platformSpiCsEnter
0083f82c   Osal_platformSpiCsExit
0084d1e0   PHYREG_read
0084ac00   PHYREG_wait
0084a1a0   PHYREG_waitResults
00848ec0   PHYREG_waitResultsAck
0084c700   PHYREG_write
008331c0   PowerUpDomains
00844740   SGMII_config
0084c760   SGMII_reset
008331f0   SetDDR3PllConfig
0085ea38   TSK_idle
00838d20   UartInit
00839358   UartIsDataReady
00839394   UartIsDataReady_B
00839160   UartReadBaudRate
008391d0   UartReadBaudRate_B
00839248   UartReadData
00839274   UartReadData_B
00839078   UartSetBaudRate
008390f0   UartSetBaudRate_B
008392a4   UartWriteData
00839300   UartWriteData_B
00800000   __ASM__
0085f614   __CIOBUF_
00800090   __ISA__
008000a8   __PLAT__
008000d0   __TARG__
0085ff5c   __TI_CINIT_Base
0085ffa4   __TI_CINIT_Limit
0085ff20   __TI_Handler_Table_Base
0085ff2c   __TI_Handler_Table_Limit
UNDEFED    __TI_INITARRAY_Base
UNDEFED    __TI_INITARRAY_Limit
0085e360   __TI_STACK_END
00001000   __TI_STACK_SIZE
0085f7a4   __TI_STATIC_BASE
00000001   __TI_args_main
0084e200   __TI_decompress_none
0084e220   __TI_decompress_rle24
0085ec3c   __TI_enable_exit_profile_output
ffffffff   __TI_pprof_out_hndl
ffffffff   __TI_prof_data_size
ffffffff   __TI_prof_data_start
00849240   __TI_zero_init
008000f8   __TRDR__
ffffffff   __binit__
0083aca0   __c6xabi_divd
0084a3e0   __c6xabi_divu
00845760   __c6xabi_divul
00842320   __c6xabi_divull
0084c7c0   __c6xabi_frcmpyd_div
0084d220   __c6xabi_isinf
0084b680   __c6xabi_llshl
0084c820   __c6xabi_llshru
0084e040   __c6xabi_negll
0084aca0   __c6xabi_remu
ffffffff   __c_args__
0084e060   __cxa_atexit
0084a320   __cxa_finalize
0084e080   __cxa_ia64_exit
0084a3e0   __divu
0084aca0   __remu
0084e0a0   __xdc__init
0085e70c   __xdc__init__addr
0084d2a0   _args_main
00000000   _argsize
00846f80   _auto_init_elf
0084ad40   _c_int00
0084ade0   _cleanup
0085ec34   _cleanup_ptr
00847d40   _closefile
00859628   _ctypes_
0084a4a0   _doflush
0085ec38   _dtors_ptr
0085ea34   _ft_end
0085e360   _ftable
0085ec40   _lock
0084e0c0   _nop
0083d7e0   _printfi
0084e140   _register_lock
0084e160   _register_unlock
0085d360   _stack
0084c880   _subcull
0085d1c8   _tmpnams
0085ec44   _unlock
008483e0   _wrt_ok
0084e1c0   abort
00833c2c   app_display_linkstatus
00834b74   app_init
0085ba8c   app_mcb
00800000   app_pkt_buffer
00833c74   app_timer
0084e1e0   atexit
00849080   atoi
ffffffff   binit
00849160   close
00846db4   configSerdes
0085f480   emac_comm_dev0
0085f600   emac_comm_pcb0
00840f80   emac_config
008484e0   emac_free_chan_comm_pcb
0084b100   emac_free_macaddr
0084e240   emac_get_version
008393e0   emac_init
00845900   emac_init_queue
00846260   emac_int_service
0085a088   emac_mcb
0083a6c0   emac_open
0083f980   emac_poll
80000d98   emac_port_mode
0084c940   emac_reset
008485e0   emac_reset_queue
00841e60   emac_send
008599a8   emac_version_str
0084b980   evmI2CInit
0084a620   exit
008494e0   fflush
0083d3b8   fpgaControlUserLEDs
0083d58c   fpgaDisableEepromWriteProtect
0083d478   fpgaDisableNandWriteProtect
0083d504   fpgaDisableNorWriteProtect
0083d5d0   fpgaEnableEepromWriteProtect
0083d4c0   fpgaEnableNandWriteProtect
0083d548   fpgaEnableNorWriteProtect
0083d660   fpgaGetAMCDetect
0083d614   fpgaGetUserSwitch
0083d750   fpgaReadConfigurationRegister
0083d6a4   fpgaWriteConfigurationRegister
008432a0   fputc
0083ec40   fputs
0084d3e0   free
00847f80   fseek
80000d24   gDeviceEeprom0
80000d5c   gDeviceEeprom1
80000cb4   gDeviceNand
80000898   gDeviceNandBBlist
80000cec   gDeviceNor
0085d308   gI2cBlock
0083d320   getBoardVersion
0083d36c   getFpgaDevID
0085f7a4   hGpio
008369c0   i2cEepromMacRead
00836728   i2cEepromMacWrite
008362ac   i2cEepromRead
008364b0   i2cEepromWrite
00835fe4   i2cEepromWriteBlock
008365d0   i2cEepromWriteByteAddr
0084b2e0   lseek
008495c0   ltoa
00834e9c   main
0084b800   malloc
0084c9a0   memccpy
0084b380   memcpy
008496a0   memset
00833ae4   myStartupFxn
00835cb8   nandFlashBlockErase
00835f80   nandInit
0083ccf4   nor_erase
0083c980   nor_get_details
0083ca0c   nor_init
0083ca90   nor_read
0083cb20   nor_write
00833ac0   phyInit
0085f7b4   pktbuf_extmem
00831748   platform_blocknpage_to_offset
00830ca0   platform_delay
00830d00   platform_delaycycles
008311d0   platform_device_close
00831d6c   platform_device_erase_block
0083130c   platform_device_mark_block_bad
0083104c   platform_device_open
008314c0   platform_device_read
0083126c   platform_device_read_spare_data
00831840   platform_device_write
00831420   platform_device_write_spare_data
0085f7ac   platform_errno
00830d40   platform_external_memory_test
00830c34   platform_fpgaReadConfigReg
00830c10   platform_fpgaWriteConfigReg
008309c4   platform_get_coreid
008309d0   platform_get_emac_info
00830af4   platform_get_emac_start_evt_id
008304a8   platform_get_info
00830a64   platform_get_macaddr
00830af8   platform_get_phy_addr
00830b18   platform_get_switch_state
008307b4   platform_init
0085f7b0   platform_init_return_code
00830dc0   platform_internal_memory_test
00830c54   platform_led
00831620   platform_offset_to_blocknpage
00830b28   platform_phy_link_status
00830bf4   platform_uart_init
00830b38   platform_uart_read
00830bc0   platform_uart_set_baudrate
00830ba4   platform_uart_write
00830f28   platform_write
00830ef0   platform_write_configure
00849780   printf
00832d24   prog_pll1_values
0084e280   putc
0084e2a0   putchar
008355e8   readNandPage
00833a08   readPhyReg
0084b880   readmsg
0084c380   remove
00830390   serial_num_isvalid
00844540   setvbuf
0083b850   spi_claim
0083bb48   spi_cmd
0083bbc0   spi_cmd_read
0083bc20   spi_cmd_write
0083bc80   spi_read_word
0083b9f8   spi_release
0083bd2c   spi_write_word
0083ba10   spi_xfer
0084d520   strlen
0084ca00   strncmp
0084b900   strncpy
008599a4   ti_sysbios_BIOS_Module__diagsEnabled__C
00859ce4   ti_sysbios_BIOS_Module__diagsIncluded__C
00859d94   ti_sysbios_BIOS_Module__diagsMask__C
0085a018   ti_sysbios_BIOS_Module__id__C
0085e540   ti_sysbios_BIOS_Module__state__V
0084e2c0   ti_sysbios_BIOS_RtsGateProxy_enter__E
0084e2e0   ti_sysbios_BIOS_RtsGateProxy_leave__E
0084a6e0   ti_sysbios_BIOS_errorRaiseHook__I
0084ca60   ti_sysbios_BIOS_exitFunc__I
00859dcc   ti_sysbios_BIOS_installedErrorHook__C
0084cac0   ti_sysbios_BIOS_registerRTSLock__I
0084e300   ti_sysbios_BIOS_setThreadType__E
0084d560   ti_sysbios_BIOS_startFunc__I
0084d5a0   ti_sysbios_BIOS_start__E
0084e320   ti_sysbios_family_c62_TaskSupport_Module__startupDone__S
0084d320   ti_sysbios_family_c62_TaskSupport_buildTaskStack
0084e340   ti_sysbios_family_c62_TaskSupport_checkStack__E
0084e360   ti_sysbios_family_c62_TaskSupport_getStackAlignment__E
0084e180   ti_sysbios_family_c62_TaskSupport_glue
00859dd8   ti_sysbios_family_c62_TaskSupport_stackAlignment__C
0084ba00   ti_sysbios_family_c62_TaskSupport_start__E
0084b700   ti_sysbios_family_c62_TaskSupport_swap__E
00859ddc   ti_sysbios_family_c64p_Exception_E_exceptionMin__C
0085a01c   ti_sysbios_family_c64p_Exception_Module__id__C
0085e55c   ti_sysbios_family_c64p_Exception_Module__state__V
0084e380   ti_sysbios_family_c64p_Exception_Module_startup__E
0084ba80   ti_sysbios_family_c64p_Exception_Module_startup__F
00846560   ti_sysbios_family_c64p_Exception_dispatch__E
00859de0   ti_sysbios_family_c64p_Exception_exceptionHook__C
00859de4   ti_sysbios_family_c64p_Exception_externalHook__C
00837ea0   ti_sysbios_family_c64p_Exception_handler__I
008429e0   ti_sysbios_family_c64p_Exception_internalHandler__I
00859de8   ti_sysbios_family_c64p_Exception_internalHook__C
00859dec   ti_sysbios_family_c64p_Exception_nmiHook__C
0085f800   ti_sysbios_family_c64p_Hwi0
0085f820   ti_sysbios_family_c64p_Hwi1
0085f940   ti_sysbios_family_c64p_Hwi10
0085f960   ti_sysbios_family_c64p_Hwi11
0085f980   ti_sysbios_family_c64p_Hwi12
0085f9a0   ti_sysbios_family_c64p_Hwi13
0085f9c0   ti_sysbios_family_c64p_Hwi14
0085f9e0   ti_sysbios_family_c64p_Hwi15
0085f840   ti_sysbios_family_c64p_Hwi2
0085f860   ti_sysbios_family_c64p_Hwi3
0085f880   ti_sysbios_family_c64p_Hwi4
0085f8a0   ti_sysbios_family_c64p_Hwi5
0085f8c0   ti_sysbios_family_c64p_Hwi6
0085f8e0   ti_sysbios_family_c64p_Hwi7
0085f900   ti_sysbios_family_c64p_Hwi8
0085f920   ti_sysbios_family_c64p_Hwi9
00859df0   ti_sysbios_family_c64p_Hwi_E_alreadyDefined__C
00859df4   ti_sysbios_family_c64p_Hwi_E_handleNotFound__C
00849860   ti_sysbios_family_c64p_Hwi_Instance_finalize__F
00849940   ti_sysbios_family_c64p_Hwi_Instance_init__F
00859df8   ti_sysbios_family_c64p_Hwi_LD_end__C
00859dfc   ti_sysbios_family_c64p_Hwi_LM_begin__C
00859e00   ti_sysbios_family_c64p_Hwi_Module__diagsEnabled__C
00859e04   ti_sysbios_family_c64p_Hwi_Module__diagsIncluded__C
00859e08   ti_sysbios_family_c64p_Hwi_Module__diagsMask__C
0085a020   ti_sysbios_family_c64p_Hwi_Module__id__C
0085a024   ti_sysbios_family_c64p_Hwi_Module__loggerDefined__C
00859e0c   ti_sysbios_family_c64p_Hwi_Module__loggerFxn1__C
00859e10   ti_sysbios_family_c64p_Hwi_Module__loggerFxn8__C
00859e14   ti_sysbios_family_c64p_Hwi_Module__loggerObj__C
0085e588   ti_sysbios_family_c64p_Hwi_Module__root__V
0084d5e0   ti_sysbios_family_c64p_Hwi_Module__startupDone__F
0084e3a0   ti_sysbios_family_c64p_Hwi_Module__startupDone__S
0085e590   ti_sysbios_family_c64p_Hwi_Module__state__V
0084e3c0   ti_sysbios_family_c64p_Hwi_Module_startup__E
008475c0   ti_sysbios_family_c64p_Hwi_Module_startup__F
00859ba4   ti_sysbios_family_c64p_Hwi_Object__DESC__C
00859974   ti_sysbios_family_c64p_Hwi_Object__PARAMS__C
00849a20   ti_sysbios_family_c64p_Hwi_Object__create__S
0084d620   ti_sysbios_family_c64p_Hwi_Object__delete__S
0085ec08   ti_sysbios_family_c64p_Hwi_Object__table__V
0084e3e0   ti_sysbios_family_c64p_Hwi_clearInterrupt__E
0084d660   ti_sysbios_family_c64p_Hwi_disableInterrupt__E
00844140   ti_sysbios_family_c64p_Hwi_dispatchAlways
0083fc80   ti_sysbios_family_c64p_Hwi_dispatchC__I
0084d6a0   ti_sysbios_family_c64p_Hwi_enableInterrupt__E
0084bb00   ti_sysbios_family_c64p_Hwi_eventMap__E
0084b060   ti_sysbios_family_c64p_Hwi_plug__E
008434c0   ti_sysbios_family_c64p_Hwi_reconfig__E
0084e400   ti_sysbios_family_c64p_Hwi_startup__E
0084e420   ti_sysbios_family_c64p_Hwi_switchFromBootStack__E
0084e440   ti_sysbios_family_c64p_Hwi_unPluggedInterrupt__I
0084e460   ti_sysbios_family_c64p_tci6488_TimerSupport_enable__E
0084e480   ti_sysbios_family_c66_Cache_Module_startup__E
00847700   ti_sysbios_family_c66_Cache_Module_startup__F
00859e18   ti_sysbios_family_c66_Cache_atomicBlockSize__C
00859d74   ti_sysbios_family_c66_Cache_initSize__C
0084bb80   ti_sysbios_family_c66_Cache_invL1pAll__E
00859228   ti_sysbios_family_c66_Cache_marvalues__C
0084e4a0   ti_sysbios_family_c66_Cache_wbInv__E
0084d360   ti_sysbios_family_xxx_Hwi_switchToIsrStack
0084e1a0   ti_sysbios_family_xxx_Hwi_switchToTaskStack
0084d6e0   ti_sysbios_gates_GateHwi_Handle__label__S
0084e4c0   ti_sysbios_gates_GateHwi_Instance_init__F
00859ad0   ti_sysbios_gates_GateHwi_Module__FXNS__C
0085e5f8   ti_sysbios_gates_GateHwi_Module__root__V
00859bc4   ti_sysbios_gates_GateHwi_Object__DESC__C
00859d00   ti_sysbios_gates_GateHwi_Object__PARAMS__C
0084bc00   ti_sysbios_gates_GateHwi_Object__create__S
0084d720   ti_sysbios_gates_GateHwi_Object__delete__S
0085ec58   ti_sysbios_gates_GateHwi_Object__table__V
0084e4e0   ti_sysbios_gates_GateHwi_enter__E
0084e500   ti_sysbios_gates_GateHwi_leave__E
0084e520   ti_sysbios_gates_GateHwi_query__E
0084e540   ti_sysbios_gates_GateHwi_query__F
00859e1c   ti_sysbios_gates_GateMutex_A_badContext__C
0084d760   ti_sysbios_gates_GateMutex_Handle__label__S
00859e20   ti_sysbios_gates_GateMutex_Instance_State_sem__O
0084d7a0   ti_sysbios_gates_GateMutex_Instance_finalize__F
0084cb20   ti_sysbios_gates_GateMutex_Instance_init__F
00859af4   ti_sysbios_gates_GateMutex_Module__FXNS__C
00859e24   ti_sysbios_gates_GateMutex_Module__diagsEnabled__C
00859e28   ti_sysbios_gates_GateMutex_Module__diagsIncluded__C
00859e2c   ti_sysbios_gates_GateMutex_Module__diagsMask__C
0085a028   ti_sysbios_gates_GateMutex_Module__id__C
0085e600   ti_sysbios_gates_GateMutex_Module__root__V
00859be4   ti_sysbios_gates_GateMutex_Object__DESC__C
00859d18   ti_sysbios_gates_GateMutex_Object__PARAMS__C
0084bc80   ti_sysbios_gates_GateMutex_Object__create__S
0084d7e0   ti_sysbios_gates_GateMutex_Object__delete__S
0085ea80   ti_sysbios_gates_GateMutex_Object__table__V
00845aa0   ti_sysbios_gates_GateMutex_enter__E
0084d820   ti_sysbios_gates_GateMutex_leave__E
0084e560   ti_sysbios_gates_GateMutex_query__E
0084e580   ti_sysbios_gates_GateMutex_query__F
00859e30   ti_sysbios_hal_Hwi_E_stackOverflow__C
0084e5a0   ti_sysbios_hal_Hwi_HwiProxy_Module__startupDone__S
0084d860   ti_sysbios_hal_Hwi_HwiProxy_Object__create__S
0084e5c0   ti_sysbios_hal_Hwi_HwiProxy_Object__delete__S
0084e5e0   ti_sysbios_hal_Hwi_HwiProxy_clearInterrupt__E
0084e600   ti_sysbios_hal_Hwi_HwiProxy_disableInterrupt__E
0084e620   ti_sysbios_hal_Hwi_HwiProxy_enableInterrupt__E
0084e640   ti_sysbios_hal_Hwi_HwiProxy_startup__E
0084e660   ti_sysbios_hal_Hwi_HwiProxy_switchFromBootStack__E
0084d8a0   ti_sysbios_hal_Hwi_Instance_finalize__F
0084cb80   ti_sysbios_hal_Hwi_Instance_init__F
0085a02c   ti_sysbios_hal_Hwi_Module__id__C
0085e608   ti_sysbios_hal_Hwi_Module__root__V
0084e680   ti_sysbios_hal_Hwi_Module_startup__E
0084e6a0   ti_sysbios_hal_Hwi_Module_startup__F
00859c04   ti_sysbios_hal_Hwi_Object__DESC__C
00859a04   ti_sysbios_hal_Hwi_Object__PARAMS__C
00849b00   ti_sysbios_hal_Hwi_Object__create__S
0085ec48   ti_sysbios_hal_Hwi_Object__table__V
0084d8e0   ti_sysbios_hal_Hwi_Params__init__S
0084bd00   ti_sysbios_hal_Hwi_checkStack
0084e5e0   ti_sysbios_hal_Hwi_clearInterrupt__E
0084e600   ti_sysbios_hal_Hwi_disableInterrupt__E
0084e620   ti_sysbios_hal_Hwi_enableInterrupt__E
0084cbe0   ti_sysbios_hal_Hwi_initStack
0084e640   ti_sysbios_hal_Hwi_startup__E
0084e660   ti_sysbios_hal_Hwi_switchFromBootStack__E
0085e610   ti_sysbios_hal_Timer_Module__root__V
0084d920   ti_sysbios_hal_Timer_Module__startupDone__F
0084e6c0   ti_sysbios_hal_Timer_Module__startupDone__S
0084e6e0   ti_sysbios_hal_Timer_Module_startup__E
0084e700   ti_sysbios_hal_Timer_Module_startup__F
0085ec50   ti_sysbios_hal_Timer_Object__table__V
0084e720   ti_sysbios_hal_Timer_TimerProxy_Module__startupDone__S
0084e740   ti_sysbios_hal_Timer_TimerProxy_getExpiredCounts__E
0084e760   ti_sysbios_hal_Timer_TimerProxy_getPeriod__E
0084e780   ti_sysbios_hal_Timer_TimerProxy_setNextTick__E
0084e7a0   ti_sysbios_hal_Timer_TimerProxy_startup__E
0084e7a0   ti_sysbios_hal_Timer_startup__E
00859e34   ti_sysbios_heaps_HeapMem_A_align__C
00859e38   ti_sysbios_heaps_HeapMem_A_heapSize__C
00859e3c   ti_sysbios_heaps_HeapMem_A_invalidFree__C
00859e40   ti_sysbios_heaps_HeapMem_A_zeroBlock__C
00859e44   ti_sysbios_heaps_HeapMem_E_memory__C
0084d960   ti_sysbios_heaps_HeapMem_Handle__label__S
0084ef80   ti_sysbios_heaps_HeapMem_Instance_State_0_buf__A
008466e0   ti_sysbios_heaps_HeapMem_Instance_init__F
0084e7c0   ti_sysbios_heaps_HeapMem_Module_GateProxy_enter__E
0084e7e0   ti_sysbios_heaps_HeapMem_Module_GateProxy_leave__E
0084e800   ti_sysbios_heaps_HeapMem_Module_GateProxy_query__E
00859a80   ti_sysbios_heaps_HeapMem_Module__FXNS__C
00859e48   ti_sysbios_heaps_HeapMem_Module__diagsEnabled__C
00859e4c   ti_sysbios_heaps_HeapMem_Module__diagsIncluded__C
00859e50   ti_sysbios_heaps_HeapMem_Module__diagsMask__C
00859e54   ti_sysbios_heaps_HeapMem_Module__gateObj__C
0085a030   ti_sysbios_heaps_HeapMem_Module__id__C
0085e618   ti_sysbios_heaps_HeapMem_Module__root__V
00859c24   ti_sysbios_heaps_HeapMem_Object__DESC__C
00859c44   ti_sysbios_heaps_HeapMem_Object__PARAMS__C
00859e58   ti_sysbios_heaps_HeapMem_Object__count__C
0084bd80   ti_sysbios_heaps_HeapMem_Object__create__S
0084d9a0   ti_sysbios_heaps_HeapMem_Object__delete__S
0084cc40   ti_sysbios_heaps_HeapMem_Object__get__S
00859e5c   ti_sysbios_heaps_HeapMem_Object__table__C
0085ec20   ti_sysbios_heaps_HeapMem_Object__table__V
0083a0a0   ti_sysbios_heaps_HeapMem_alloc__E
00839a40   ti_sysbios_heaps_HeapMem_free__E
0084a7a0   ti_sysbios_heaps_HeapMem_getStats__E
0084b420   ti_sysbios_heaps_HeapMem_init__I
0084e820   ti_sysbios_heaps_HeapMem_isBlocking__E
00859e60   ti_sysbios_heaps_HeapMem_reqAlignMask__C
00859e64   ti_sysbios_heaps_HeapMem_reqAlign__C
00859e68   ti_sysbios_knl_Clock_A_badThreadType__C
00847840   ti_sysbios_knl_Clock_Instance_finalize__F
00841200   ti_sysbios_knl_Clock_Instance_init__F
00859e6c   ti_sysbios_knl_Clock_LM_begin__C
00859e70   ti_sysbios_knl_Clock_LM_tick__C
00859e74   ti_sysbios_knl_Clock_LW_delayed__C
00859e78   ti_sysbios_knl_Clock_Module_State_clockQ__O
00859e7c   ti_sysbios_knl_Clock_Module__diagsEnabled__C
00859e80   ti_sysbios_knl_Clock_Module__diagsIncluded__C
00859e84   ti_sysbios_knl_Clock_Module__diagsMask__C
0085a034   ti_sysbios_knl_Clock_Module__id__C
0085a038   ti_sysbios_knl_Clock_Module__loggerDefined__C
00859e88   ti_sysbios_knl_Clock_Module__loggerFxn1__C
00859e8c   ti_sysbios_knl_Clock_Module__loggerFxn2__C
00859e90   ti_sysbios_knl_Clock_Module__loggerObj__C
0085e620   ti_sysbios_knl_Clock_Module__root__V
0085e628   ti_sysbios_knl_Clock_Module__state__V
0084e860   ti_sysbios_knl_Clock_Module_startup__E
0084be00   ti_sysbios_knl_Clock_Module_startup__F
00859c64   ti_sysbios_knl_Clock_Object__DESC__C
00859b18   ti_sysbios_knl_Clock_Object__PARAMS__C
0084be80   ti_sysbios_knl_Clock_Object__create__S
0084d9e0   ti_sysbios_knl_Clock_Object__destruct__S
0085ebb0   ti_sysbios_knl_Clock_Object__table__V
0084da20   ti_sysbios_knl_Clock_Params__init__S
0084cca0   ti_sysbios_knl_Clock_doTick__I
0084bf00   ti_sysbios_knl_Clock_getTicks__E
0084a860   ti_sysbios_knl_Clock_logTick__E
008487e0   ti_sysbios_knl_Clock_startI__E
00849be0   ti_sysbios_knl_Clock_start__E
00859e94   ti_sysbios_knl_Clock_tickMode__C
00859e98   ti_sysbios_knl_Clock_tickSource__C
008407e0   ti_sysbios_knl_Clock_workFunc__E
00859ea0   ti_sysbios_knl_Idle_funcList__A
00859dac   ti_sysbios_knl_Idle_funcList__C
0084bf80   ti_sysbios_knl_Idle_loop__E
0084e880   ti_sysbios_knl_Queue_Instance_init__F
0085e654   ti_sysbios_knl_Queue_Module__root__V
00859c84   ti_sysbios_knl_Queue_Object__DESC__C
00859d30   ti_sysbios_knl_Queue_Object__PARAMS__C
00859e9c   ti_sysbios_knl_Queue_Object__count__C
0084c000   ti_sysbios_knl_Queue_Object__create__S
0084da60   ti_sysbios_knl_Queue_Object__destruct__S
0084cd00   ti_sysbios_knl_Queue_Object__get__S
00859ea4   ti_sysbios_knl_Queue_Object__table__C
0084e8a0   ti_sysbios_knl_Queue_empty__E
00859ea8   ti_sysbios_knl_Semaphore_A_badContext__C
00859eac   ti_sysbios_knl_Semaphore_A_noEvents__C
00859eb0   ti_sysbios_knl_Semaphore_A_overflow__C
00859eb4   ti_sysbios_knl_Semaphore_Instance_State_pendQ__O
0084daa0   ti_sysbios_knl_Semaphore_Instance_finalize__F
00847980   ti_sysbios_knl_Semaphore_Instance_init__F
00859eb8   ti_sysbios_knl_Semaphore_LM_pend__C
00859ebc   ti_sysbios_knl_Semaphore_LM_post__C
00859ec0   ti_sysbios_knl_Semaphore_Module__diagsEnabled__C
00859ec4   ti_sysbios_knl_Semaphore_Module__diagsIncluded__C
00859ec8   ti_sysbios_knl_Semaphore_Module__diagsMask__C
0085a03c   ti_sysbios_knl_Semaphore_Module__id__C
0085a040   ti_sysbios_knl_Semaphore_Module__loggerDefined__C
00859ecc   ti_sysbios_knl_Semaphore_Module__loggerFxn2__C
00859ed0   ti_sysbios_knl_Semaphore_Module__loggerFxn4__C
00859ed4   ti_sysbios_knl_Semaphore_Module__loggerObj__C
0085e65c   ti_sysbios_knl_Semaphore_Module__root__V
00859ca4   ti_sysbios_knl_Semaphore_Object__DESC__C
00859b3c   ti_sysbios_knl_Semaphore_Object__PARAMS__C
0084c080   ti_sysbios_knl_Semaphore_Object__create__S
0084dae0   ti_sysbios_knl_Semaphore_Object__destruct__S
0084c100   ti_sysbios_knl_Semaphore_pendTimeout__I
0083e0a0   ti_sysbios_knl_Semaphore_pend__E
00842c20   ti_sysbios_knl_Semaphore_post__E
00859ed8   ti_sysbios_knl_Swi_LD_end__C
00859edc   ti_sysbios_knl_Swi_LM_begin__C
00859ee0   ti_sysbios_knl_Swi_LM_post__C
0085e870   ti_sysbios_knl_Swi_Module_State_0_readyQ__A
00859ee4   ti_sysbios_knl_Swi_Module__diagsEnabled__C
00859ee8   ti_sysbios_knl_Swi_Module__diagsIncluded__C
00859eec   ti_sysbios_knl_Swi_Module__diagsMask__C
0085a044   ti_sysbios_knl_Swi_Module__id__C
0085a048   ti_sysbios_knl_Swi_Module__loggerDefined__C
00859ef0   ti_sysbios_knl_Swi_Module__loggerFxn1__C
00859ef4   ti_sysbios_knl_Swi_Module__loggerFxn4__C
00859ef8   ti_sysbios_knl_Swi_Module__loggerObj__C
0085e664   ti_sysbios_knl_Swi_Module__root__V
0085e66c   ti_sysbios_knl_Swi_Module__state__V
0084e8c0   ti_sysbios_knl_Swi_Module_startup__E
0084cd60   ti_sysbios_knl_Swi_Module_startup__F
00859efc   ti_sysbios_knl_Swi_Object__count__C
0084cdc0   ti_sysbios_knl_Swi_Object__get__S
00859f00   ti_sysbios_knl_Swi_Object__table__C
0085eb80   ti_sysbios_knl_Swi_Object__table__V
0084e8e0   ti_sysbios_knl_Swi_disable__E
00847ac0   ti_sysbios_knl_Swi_post__E
008488e0   ti_sysbios_knl_Swi_restoreHwi__E
008436e0   ti_sysbios_knl_Swi_run__I
00846860   ti_sysbios_knl_Swi_schedule__I
0084c180   ti_sysbios_knl_Swi_startup__E
00859f04   ti_sysbios_knl_Task_A_badPriority__C
00859f08   ti_sysbios_knl_Task_A_badTaskState__C
00859f0c   ti_sysbios_knl_Task_A_badThreadType__C
00859f10   ti_sysbios_knl_Task_A_noPendElem__C
00859f14   ti_sysbios_knl_Task_E_spOutOfBounds__C
00859f18   ti_sysbios_knl_Task_E_stackOverflow__C
0085d358   ti_sysbios_knl_Task_Instance_State_0_hookEnv__A
0085ec60   ti_sysbios_knl_Task_Instance_State_0_stack__A
0083ce20   ti_sysbios_knl_Task_Instance_finalize__F
0083e880   ti_sysbios_knl_Task_Instance_init__F
00859f1c   ti_sysbios_knl_Task_LD_block__C
00859f20   ti_sysbios_knl_Task_LD_exit__C
00859f24   ti_sysbios_knl_Task_LD_ready__C
00859f28   ti_sysbios_knl_Task_LM_switch__C
0085e8f0   ti_sysbios_knl_Task_Module_State_0_readyQ__A
00859f2c   ti_sysbios_knl_Task_Module_State_inactiveQ__O
00859f30   ti_sysbios_knl_Task_Module_State_terminatedQ__O
00859f34   ti_sysbios_knl_Task_Module__diagsEnabled__C
00859f38   ti_sysbios_knl_Task_Module__diagsIncluded__C
00859f3c   ti_sysbios_knl_Task_Module__diagsMask__C
0085a04c   ti_sysbios_knl_Task_Module__id__C
0085a050   ti_sysbios_knl_Task_Module__loggerDefined__C
00859f40   ti_sysbios_knl_Task_Module__loggerFxn2__C
00859f44   ti_sysbios_knl_Task_Module__loggerFxn4__C
00859f48   ti_sysbios_knl_Task_Module__loggerObj__C
0085e688   ti_sysbios_knl_Task_Module__root__V
0085e690   ti_sysbios_knl_Task_Module__state__V
0084e900   ti_sysbios_knl_Task_Module_startup__E
00840260   ti_sysbios_knl_Task_Module_startup__F
00859cc4   ti_sysbios_knl_Task_Object__DESC__C
0085993c   ti_sysbios_knl_Task_Object__PARAMS__C
00859f4c   ti_sysbios_knl_Task_Object__count__C
0084a920   ti_sysbios_knl_Task_Object__create__S
0084db20   ti_sysbios_knl_Task_Object__first__S
0084ce20   ti_sysbios_knl_Task_Object__get__S
00859f50   ti_sysbios_knl_Task_Object__heap__C
0084db60   ti_sysbios_knl_Task_Object__next__S
00859f54   ti_sysbios_knl_Task_Object__table__C
0085ea38   ti_sysbios_knl_Task_Object__table__V
0084dba0   ti_sysbios_knl_Task_Params__init__S
0084e920   ti_sysbios_knl_Task_SupportProxy_Module__startupDone__S
0084e940   ti_sysbios_knl_Task_SupportProxy_checkStack__E
0084e960   ti_sysbios_knl_Task_SupportProxy_getStackAlignment__E
0084e980   ti_sysbios_knl_Task_SupportProxy_start__E
0084e9a0   ti_sysbios_knl_Task_SupportProxy_swap__E
00859f58   ti_sysbios_knl_Task_allBlockedFunc__C
0084ce80   ti_sysbios_knl_Task_allBlockedFunction__I
00847c00   ti_sysbios_knl_Task_blockI__E
00845240   ti_sysbios_knl_Task_checkStacks__E
00859f5c   ti_sysbios_knl_Task_defaultStackHeap__C
00859f60   ti_sysbios_knl_Task_defaultStackSize__C
0085a054   ti_sysbios_knl_Task_deleteTerminatedTasks__C
0084e9c0   ti_sysbios_knl_Task_disable__E
0084cee0   ti_sysbios_knl_Task_enter__I
00841480   ti_sysbios_knl_Task_exit__E
00859d48   ti_sysbios_knl_Task_hooks__A
00859db4   ti_sysbios_knl_Task_hooks__C
0085a058   ti_sysbios_knl_Task_initStackFlag__C
00859f64   ti_sysbios_knl_Task_numConstructedTasks__C
00859f68   ti_sysbios_knl_Task_numPriorities__C
00844b00   ti_sysbios_knl_Task_postInit__I
0084c200   ti_sysbios_knl_Task_restore__E
00843900   ti_sysbios_knl_Task_schedule__I
00843b20   ti_sysbios_knl_Task_startup__E
008469e0   ti_sysbios_knl_Task_unblockI__E
00859f6c   ti_sysbios_timers_timer64_Timer_A_notAvailable__C
00859f70   ti_sysbios_timers_timer64_Timer_E_cannotSupport__C
0085e710   ti_sysbios_timers_timer64_Timer_Module_State_0_device__A
0085eac0   ti_sysbios_timers_timer64_Timer_Module_State_0_gctrl__A
0085eb00   ti_sysbios_timers_timer64_Timer_Module_State_0_handles__A
0085eb40   ti_sysbios_timers_timer64_Timer_Module_State_0_intFreqs__A
00859f74   ti_sysbios_timers_timer64_Timer_Module__diagsEnabled__C
00859f78   ti_sysbios_timers_timer64_Timer_Module__diagsIncluded__C
00859f7c   ti_sysbios_timers_timer64_Timer_Module__diagsMask__C
0085a05c   ti_sysbios_timers_timer64_Timer_Module__id__C
0085e6c4   ti_sysbios_timers_timer64_Timer_Module__root__V
0084dbe0   ti_sysbios_timers_timer64_Timer_Module__startupDone__F
0084e9e0   ti_sysbios_timers_timer64_Timer_Module__startupDone__S
0085e6cc   ti_sysbios_timers_timer64_Timer_Module__state__V
0084ea00   ti_sysbios_timers_timer64_Timer_Module_startup__E
0083bde0   ti_sysbios_timers_timer64_Timer_Module_startup__F
0085e9e8   ti_sysbios_timers_timer64_Timer_Object__table__V
0084ea20   ti_sysbios_timers_timer64_Timer_TimerSupportProxy_enable__E
00859f80   ti_sysbios_timers_timer64_Timer_anyMask__C
00859f84   ti_sysbios_timers_timer64_Timer_freqDivisor__C
0084c280   ti_sysbios_timers_timer64_Timer_getCount__E
0084c280   ti_sysbios_timers_timer64_Timer_getExpiredCounts__E
00844ce0   ti_sysbios_timers_timer64_Timer_getFreq__E
0084c300   ti_sysbios_timers_timer64_Timer_getPeriod__E
00859f88   ti_sysbios_timers_timer64_Timer_numLocalTimers__C
00859f8c   ti_sysbios_timers_timer64_Timer_numTimerDevices__C
0084ea40   ti_sysbios_timers_timer64_Timer_setNextTick__E
00845400   ti_sysbios_timers_timer64_Timer_setPeriodMicroSecs__E
00845c40   ti_sysbios_timers_timer64_Timer_start__E
0085a060   ti_sysbios_timers_timer64_Timer_startupNeeded__C
00849cc0   ti_sysbios_timers_timer64_Timer_startup__E
0084a9e0   ti_sysbios_timers_timer64_Timer_stop__E
0084c380   unlink
0084cf40   vsprintf
0084b4c0   write
00835914   writeNandPage
00833a64   writePhyReg
0084cfa0   writemsg
00859f90   xdc_runtime_Assert_E_assertFailed__C
0084b560   xdc_runtime_Assert_raise__I
00859f94   xdc_runtime_Core_A_initializedParams__C
00859f98   xdc_runtime_Core_Module__diagsEnabled__C
00859f9c   xdc_runtime_Core_Module__diagsIncluded__C
00859fa0   xdc_runtime_Core_Module__diagsMask__C
0085a064   xdc_runtime_Core_Module__id__C
0084c400   xdc_runtime_Core_assignLabel__I
0084c480   xdc_runtime_Core_assignParams__I
00841700   xdc_runtime_Core_createObject__I
008489e0   xdc_runtime_Core_deleteObject__I
00859fa4   xdc_runtime_Error_E_generic__C
00859fa8   xdc_runtime_Error_E_memory__C
00859fac   xdc_runtime_Error_Module__diagsEnabled__C
00859fb0   xdc_runtime_Error_Module__diagsIncluded__C
00859fb4   xdc_runtime_Error_Module__diagsMask__C
0085a068   xdc_runtime_Error_Module__loggerDefined__C
00859fb8   xdc_runtime_Error_Module__loggerFxn8__C
00859fbc   xdc_runtime_Error_Module__loggerObj__C
0085e6e0   xdc_runtime_Error_Module__state__V
0084ea80   xdc_runtime_Error_check__E
0084dc20   xdc_runtime_Error_check__F
0084eaa0   xdc_runtime_Error_init__E
0084dc60   xdc_runtime_Error_init__F
0085a06c   xdc_runtime_Error_maxDepth__C
00859fc0   xdc_runtime_Error_policy__C
0084eac0   xdc_runtime_Error_print__E
00849da0   xdc_runtime_Error_print__F
00859fc4   xdc_runtime_Error_raiseHook__C
0084dca0   xdc_runtime_Error_raiseX__E
00841980   xdc_runtime_Error_raiseX__F
0084eae0   xdc_runtime_Gate_enterSystem__E
0084eb00   xdc_runtime_Gate_enterSystem__F
0084eb20   xdc_runtime_Gate_leaveSystem__E
0084dce0   xdc_runtime_Gate_leaveSystem__F
00859fc8   xdc_runtime_IGateProvider_Interface__BASE__C
00859fcc   xdc_runtime_IHeap_Interface__BASE__C
00859fd0   xdc_runtime_IModule_Interface__BASE__C
00859fd4   xdc_runtime_Log_L_error__C
0084eb40   xdc_runtime_Memory_HeapProxy_alloc__E
0084eb60   xdc_runtime_Memory_HeapProxy_free__E
0085a070   xdc_runtime_Memory_Module__id__C
0085e6e4   xdc_runtime_Memory_Module__state__V
0084eb80   xdc_runtime_Memory_alloc__E
00849e80   xdc_runtime_Memory_alloc__F
0084eba0   xdc_runtime_Memory_calloc__E
0084d000   xdc_runtime_Memory_calloc__F
00859fd8   xdc_runtime_Memory_defaultHeapInstance__C
0084ebc0   xdc_runtime_Memory_free__E
0084dda0   xdc_runtime_Memory_free__F
0085e6e8   xdc_runtime_Registry_Module__state__V
0084ebe0   xdc_runtime_Registry_findById__E
0084dde0   xdc_runtime_Registry_findById__F
0085e6f0   xdc_runtime_Startup_Module__state__V
00000001   xdc_runtime_Startup__EXECFXN__C
00000001   xdc_runtime_Startup__RESETFXN__C
00859fdc   xdc_runtime_Startup_execImpl__C
0084ec00   xdc_runtime_Startup_exec__E
00848ae0   xdc_runtime_Startup_exec__F
0084de20   xdc_runtime_Startup_exec__I
00859d98   xdc_runtime_Startup_firstFxns__A
00859dbc   xdc_runtime_Startup_firstFxns__C
00859fe0   xdc_runtime_Startup_lastFxns__A
00859dc4   xdc_runtime_Startup_lastFxns__C
00859fe4   xdc_runtime_Startup_maxPasses__C
0084ec20   xdc_runtime_Startup_reset__I
00859d60   xdc_runtime_Startup_sfxnRts__A
00859fe8   xdc_runtime_Startup_sfxnRts__C
00859aa8   xdc_runtime_Startup_sfxnTab__A
00859fec   xdc_runtime_Startup_sfxnTab__C
00859ff0   xdc_runtime_Startup_startModsFxn__C
008420c0   xdc_runtime_Startup_startMods__I
0084ec40   xdc_runtime_SysStd_abort__E
0084d060   xdc_runtime_SysStd_abort__F
0084ec60   xdc_runtime_SysStd_exit__E
0084ec80   xdc_runtime_SysStd_exit__F
0084eca0   xdc_runtime_SysStd_putch__E
0084ecc0   xdc_runtime_SysStd_putch__F
0084ece0   xdc_runtime_SysStd_ready__E
0084ed00   xdc_runtime_SysStd_ready__F
0084ed20   xdc_runtime_System_Module_GateProxy_enter__E
0084ed40   xdc_runtime_System_Module_GateProxy_leave__E
0085ebd0   xdc_runtime_System_Module_State_0_atexitHandlers__A
00859ff4   xdc_runtime_System_Module__gateObj__C
0085e6f8   xdc_runtime_System_Module__state__V
0084ed60   xdc_runtime_System_Module_startup__E
0084ed80   xdc_runtime_System_Module_startup__F
0084eda0   xdc_runtime_System_SupportProxy_abort__E
0084edc0   xdc_runtime_System_SupportProxy_exit__E
0084ede0   xdc_runtime_System_SupportProxy_putch__E
0084ee00   xdc_runtime_System_SupportProxy_ready__E
0084ee20   xdc_runtime_System_abort__E
0084de60   xdc_runtime_System_abort__F
0084dea0   xdc_runtime_System_aprintf__E
0084d0c0   xdc_runtime_System_aprintf_va__F
0084ee40   xdc_runtime_System_atexit__E
0084c500   xdc_runtime_System_atexit__F
0084d0c0   xdc_runtime_System_avprintf__F
00836d20   xdc_runtime_System_doPrint__I
0084ee60   xdc_runtime_System_exit__E
0084ee80   xdc_runtime_System_exit__F
00859ff8   xdc_runtime_System_extendFxn__C
0084aaa0   xdc_runtime_System_formatNum__I
0084eea0   xdc_runtime_System_lastFxn__I
00859ffc   xdc_runtime_System_maxAtexitHandlers__C
0083efe0   xdc_runtime_System_printfExtend__I
0084dee0   xdc_runtime_System_printf__E
0084d120   xdc_runtime_System_printf_va__F
0084c580   xdc_runtime_System_rtsExit__I
0084eee0   xdc_runtime_System_sprintf_va__F
0084d120   xdc_runtime_System_vprintf__F
0084eec0   xdc_runtime_System_vsprintf__E
0084eee0   xdc_runtime_System_vsprintf__F
0085e704   xdc_runtime_Text_Module__state__V
0085a074   xdc_runtime_Text_charCnt__C
00856f80   xdc_runtime_Text_charTab__A
0085a000   xdc_runtime_Text_charTab__C
0084ef00   xdc_runtime_Text_cordText__E
0084d180   xdc_runtime_Text_cordText__F
0085a078   xdc_runtime_Text_isLoaded__C
0085a004   xdc_runtime_Text_nameEmpty__C
0085a008   xdc_runtime_Text_nameStatic__C
0085a00c   xdc_runtime_Text_nameUnknown__C
00859730   xdc_runtime_Text_nodeTab__A
0085a010   xdc_runtime_Text_nodeTab__C
0084c600   xdc_runtime_Text_printVisFxn__I
0084ef20   xdc_runtime_Text_putLab__E
008481c0   xdc_runtime_Text_putLab__F
00848be0   xdc_runtime_Text_putMod__F
0084ef40   xdc_runtime_Text_putSite__E
00846b60   xdc_runtime_Text_putSite__F
0085a07c   xdc_runtime_Text_registryModsLastId__C
0084ef60   xdc_runtime_Text_ropeText__E
0084df20   xdc_runtime_Text_ropeText__F
0085a080   xdc_runtime_Text_unnamedModsLastId__C
00848ce0   xdc_runtime_Text_visitRope2__I
0085a014   xdc_runtime_Text_visitRopeFxn__C
0084df60   xdc_runtime_Text_visitRope__I
0084c680   xdc_runtime_Text_xprintf__I
00833354   xmc_setup


GLOBAL SYMBOLS: SORTED BY Symbol Address 

address    name
--------   ----
00000000   _argsize
00000001   __TI_args_main
00000001   xdc_runtime_Startup__EXECFXN__C
00000001   xdc_runtime_Startup__RESETFXN__C
00001000   __TI_STACK_SIZE
00800000   __ASM__
00800000   app_pkt_buffer
00800090   __ISA__
008000a8   __PLAT__
008000d0   __TARG__
008000f8   __TRDR__
00830390   serial_num_isvalid
008304a8   platform_get_info
008307b4   platform_init
008309c4   platform_get_coreid
008309d0   platform_get_emac_info
00830a64   platform_get_macaddr
00830af4   platform_get_emac_start_evt_id
00830af8   platform_get_phy_addr
00830b18   platform_get_switch_state
00830b28   platform_phy_link_status
00830b38   platform_uart_read
00830ba4   platform_uart_write
00830bc0   platform_uart_set_baudrate
00830bf4   platform_uart_init
00830c10   platform_fpgaWriteConfigReg
00830c34   platform_fpgaReadConfigReg
00830c54   platform_led
00830ca0   platform_delay
00830d00   platform_delaycycles
00830d40   platform_external_memory_test
00830dc0   platform_internal_memory_test
00830ef0   platform_write_configure
00830f28   platform_write
0083104c   platform_device_open
008311d0   platform_device_close
0083126c   platform_device_read_spare_data
0083130c   platform_device_mark_block_bad
00831420   platform_device_write_spare_data
008314c0   platform_device_read
00831620   platform_offset_to_blocknpage
00831748   platform_blocknpage_to_offset
00831840   platform_device_write
00831d6c   platform_device_erase_block
00831e30   Convert_CoreLocal2GlobalAddr
00832d24   prog_pll1_values
00832e88   CorePllcHwSetup
008330d4   CorePllcGetHwSetup
008331c0   PowerUpDomains
008331f0   SetDDR3PllConfig
00833354   xmc_setup
008333a0   DDR3Init
00833a04   DDR2Init
00833a08   readPhyReg
00833a64   writePhyReg
00833ac0   phyInit
00833ae4   myStartupFxn
00833c2c   app_display_linkstatus
00833c74   app_timer
00834b74   app_init
00834ce0   EVM_init
00834e9c   main
008354f0   NandReadSpareArea
008355e8   readNandPage
008358b0   NandWriteDataBytes
00835914   writeNandPage
00835ba0   NandWriteSpareArea
00835cb8   nandFlashBlockErase
00835e78   NandGetDetails
00835f80   nandInit
00835fe4   i2cEepromWriteBlock
008362ac   i2cEepromRead
008364b0   i2cEepromWrite
008365d0   i2cEepromWriteByteAddr
00836728   i2cEepromMacWrite
008369c0   i2cEepromMacRead
00836d20   xdc_runtime_System_doPrint__I
008376c0   EMAC_coreInit
00837ea0   ti_sysbios_family_c64p_Exception_handler__I
00838620   MDIO_timerTick
00838d20   UartInit
00839078   UartSetBaudRate
008390f0   UartSetBaudRate_B
00839160   UartReadBaudRate
008391d0   UartReadBaudRate_B
00839248   UartReadData
00839274   UartReadData_B
008392a4   UartWriteData
00839300   UartWriteData_B
00839358   UartIsDataReady
00839394   UartIsDataReady_B
008393e0   emac_init
00839a40   ti_sysbios_heaps_HeapMem_free__E
0083a0a0   ti_sysbios_heaps_HeapMem_alloc__E
0083a6c0   emac_open
0083aca0   __c6xabi_divd
0083b850   spi_claim
0083b9f8   spi_release
0083ba10   spi_xfer
0083bb48   spi_cmd
0083bbc0   spi_cmd_read
0083bc20   spi_cmd_write
0083bc80   spi_read_word
0083bd2c   spi_write_word
0083bde0   ti_sysbios_timers_timer64_Timer_Module_startup__F
0083c3a0   EMAC_commonInit
0083c980   nor_get_details
0083ca0c   nor_init
0083ca90   nor_read
0083cb20   nor_write
0083ccf4   nor_erase
0083ce20   ti_sysbios_knl_Task_Instance_finalize__F
0083d320   getBoardVersion
0083d36c   getFpgaDevID
0083d3b8   fpgaControlUserLEDs
0083d478   fpgaDisableNandWriteProtect
0083d4c0   fpgaEnableNandWriteProtect
0083d504   fpgaDisableNorWriteProtect
0083d548   fpgaEnableNorWriteProtect
0083d58c   fpgaDisableEepromWriteProtect
0083d5d0   fpgaEnableEepromWriteProtect
0083d614   fpgaGetUserSwitch
0083d660   fpgaGetAMCDetect
0083d6a4   fpgaWriteConfigurationRegister
0083d750   fpgaReadConfigurationRegister
0083d7e0   _printfi
0083e0a0   ti_sysbios_knl_Semaphore_pend__E
0083e4a0   EMAC_coreDeInit
0083e880   ti_sysbios_knl_Task_Instance_init__F
0083ec40   fputs
0083efe0   xdc_runtime_System_printfExtend__I
0083f7b4   Osal_platformMalloc
0083f7e8   Osal_platformFree
0083f810   Osal_platformSpiCsEnter
0083f82c   Osal_platformSpiCsExit
0083f838   Osal_emacBeginMemAccess
0083f874   Osal_emacEndMemAccess
0083f8b0   Osal_emacEnterSingleCoreCriticalSection
0083f8d4   Osal_emacExitSingleCoreCriticalSection
0083f8f8   Osal_emacEnterMultipleCoreCriticalSection
0083f908   Osal_emacExitMultipleCoreCriticalSection
0083f918   Osal_emacMalloc
0083f948   Osal_emacFree
0083f980   emac_poll
0083fc80   ti_sysbios_family_c64p_Hwi_dispatchC__I
00840260   ti_sysbios_knl_Task_Module_startup__F
008407e0   ti_sysbios_knl_Clock_workFunc__E
00840f80   emac_config
00841200   ti_sysbios_knl_Clock_Instance_init__F
00841480   ti_sysbios_knl_Task_exit__E
00841700   xdc_runtime_Core_createObject__I
00841980   xdc_runtime_Error_raiseX__F
00841c00   EMAC_setMulticast
00841e60   emac_send
008420c0   xdc_runtime_Startup_startMods__I
00842320   __c6xabi_divull
008429e0   ti_sysbios_family_c64p_Exception_internalHandler__I
00842c20   ti_sysbios_knl_Semaphore_post__E
00842e60   EMAC_sendPacket
008432a0   fputc
008434c0   ti_sysbios_family_c64p_Hwi_reconfig__E
008436e0   ti_sysbios_knl_Swi_run__I
00843900   ti_sysbios_knl_Task_schedule__I
00843b20   ti_sysbios_knl_Task_startup__E
00843d40   EMAC_RxServiceCheck
00844140   ti_sysbios_family_c64p_Hwi_dispatchAlways
00844540   setvbuf
00844740   SGMII_config
00844b00   ti_sysbios_knl_Task_postInit__I
00844ce0   ti_sysbios_timers_timer64_Timer_getFreq__E
00844ec0   EMAC_TxServiceCheck
00845240   ti_sysbios_knl_Task_checkStacks__E
00845400   ti_sysbios_timers_timer64_Timer_setPeriodMicroSecs__E
008455c0   HOSTrename
00845760   __c6xabi_divul
00845900   emac_init_queue
00845aa0   ti_sysbios_gates_GateMutex_enter__E
00845c40   ti_sysbios_timers_timer64_Timer_start__E
00845de0   EMAC_setReceiveFilter
00846260   emac_int_service
00846560   ti_sysbios_family_c64p_Exception_dispatch__E
008466e0   ti_sysbios_heaps_HeapMem_Instance_init__F
00846860   ti_sysbios_knl_Swi_schedule__I
008469e0   ti_sysbios_knl_Task_unblockI__E
00846b60   xdc_runtime_Text_putSite__F
00846db4   configSerdes
00846e40   CSL_chipReadReg
00846f80   _auto_init_elf
008475c0   ti_sysbios_family_c64p_Hwi_Module_startup__F
00847700   ti_sysbios_family_c66_Cache_Module_startup__F
00847840   ti_sysbios_knl_Clock_Instance_finalize__F
00847980   ti_sysbios_knl_Semaphore_Instance_init__F
00847ac0   ti_sysbios_knl_Swi_post__E
00847c00   ti_sysbios_knl_Task_blockI__E
00847d40   _closefile
00847f80   fseek
008481c0   xdc_runtime_Text_putLab__F
008482e0   HOSTlseek
008483e0   _wrt_ok
008484e0   emac_free_chan_comm_pcb
008485e0   emac_reset_queue
008487e0   ti_sysbios_knl_Clock_startI__E
008488e0   ti_sysbios_knl_Swi_restoreHwi__E
008489e0   xdc_runtime_Core_deleteObject__I
00848ae0   xdc_runtime_Startup_exec__F
00848be0   xdc_runtime_Text_putMod__F
00848ce0   xdc_runtime_Text_visitRope2__I
00848de0   HOSTopen
00848ec0   PHYREG_waitResultsAck
00849080   atoi
00849160   close
00849240   __TI_zero_init
008494e0   fflush
008495c0   ltoa
008496a0   memset
00849780   printf
00849860   ti_sysbios_family_c64p_Hwi_Instance_finalize__F
00849940   ti_sysbios_family_c64p_Hwi_Instance_init__F
00849a20   ti_sysbios_family_c64p_Hwi_Object__create__S
00849b00   ti_sysbios_hal_Hwi_Object__create__S
00849be0   ti_sysbios_knl_Clock_start__E
00849cc0   ti_sysbios_timers_timer64_Timer_startup__E
00849da0   xdc_runtime_Error_print__F
00849e80   xdc_runtime_Memory_alloc__F
00849f60   HOSTread
0084a020   HOSTunlink
0084a0e0   HOSTwrite
0084a1a0   PHYREG_waitResults
0084a320   __cxa_finalize
0084a3e0   __c6xabi_divu
0084a3e0   __divu
0084a4a0   _doflush
0084a620   exit
0084a6e0   ti_sysbios_BIOS_errorRaiseHook__I
0084a7a0   ti_sysbios_heaps_HeapMem_getStats__E
0084a860   ti_sysbios_knl_Clock_logTick__E
0084a920   ti_sysbios_knl_Task_Object__create__S
0084a9e0   ti_sysbios_timers_timer64_Timer_stop__E
0084aaa0   xdc_runtime_System_formatNum__I
0084ab60   HOSTclose
0084ac00   PHYREG_wait
0084aca0   __c6xabi_remu
0084aca0   __remu
0084ad40   _c_int00
0084ade0   _cleanup
0084b060   ti_sysbios_family_c64p_Hwi_plug__E
0084b100   emac_free_macaddr
0084b2e0   lseek
0084b380   memcpy
0084b420   ti_sysbios_heaps_HeapMem_init__I
0084b4c0   write
0084b560   xdc_runtime_Assert_raise__I
0084b600   MDIO_open
0084b680   __c6xabi_llshl
0084b700   ti_sysbios_family_c62_TaskSupport_swap__E
0084b800   malloc
0084b880   readmsg
0084b900   strncpy
0084b980   evmI2CInit
0084ba00   ti_sysbios_family_c62_TaskSupport_start__E
0084ba80   ti_sysbios_family_c64p_Exception_Module_startup__F
0084bb00   ti_sysbios_family_c64p_Hwi_eventMap__E
0084bb80   ti_sysbios_family_c66_Cache_invL1pAll__E
0084bc00   ti_sysbios_gates_GateHwi_Object__create__S
0084bc80   ti_sysbios_gates_GateMutex_Object__create__S
0084bd00   ti_sysbios_hal_Hwi_checkStack
0084bd80   ti_sysbios_heaps_HeapMem_Object__create__S
0084be00   ti_sysbios_knl_Clock_Module_startup__F
0084be80   ti_sysbios_knl_Clock_Object__create__S
0084bf00   ti_sysbios_knl_Clock_getTicks__E
0084bf80   ti_sysbios_knl_Idle_loop__E
0084c000   ti_sysbios_knl_Queue_Object__create__S
0084c080   ti_sysbios_knl_Semaphore_Object__create__S
0084c100   ti_sysbios_knl_Semaphore_pendTimeout__I
0084c180   ti_sysbios_knl_Swi_startup__E
0084c200   ti_sysbios_knl_Task_restore__E
0084c280   ti_sysbios_timers_timer64_Timer_getCount__E
0084c280   ti_sysbios_timers_timer64_Timer_getExpiredCounts__E
0084c300   ti_sysbios_timers_timer64_Timer_getPeriod__E
0084c380   remove
0084c380   unlink
0084c400   xdc_runtime_Core_assignLabel__I
0084c480   xdc_runtime_Core_assignParams__I
0084c500   xdc_runtime_System_atexit__F
0084c580   xdc_runtime_System_rtsExit__I
0084c600   xdc_runtime_Text_printVisFxn__I
0084c680   xdc_runtime_Text_xprintf__I
0084c700   PHYREG_write
0084c760   SGMII_reset
0084c7c0   __c6xabi_frcmpyd_div
0084c820   __c6xabi_llshru
0084c880   _subcull
0084c940   emac_reset
0084c9a0   memccpy
0084ca00   strncmp
0084ca60   ti_sysbios_BIOS_exitFunc__I
0084cac0   ti_sysbios_BIOS_registerRTSLock__I
0084cb20   ti_sysbios_gates_GateMutex_Instance_init__F
0084cb80   ti_sysbios_hal_Hwi_Instance_init__F
0084cbe0   ti_sysbios_hal_Hwi_initStack
0084cc40   ti_sysbios_heaps_HeapMem_Object__get__S
0084cca0   ti_sysbios_knl_Clock_doTick__I
0084cd00   ti_sysbios_knl_Queue_Object__get__S
0084cd60   ti_sysbios_knl_Swi_Module_startup__F
0084cdc0   ti_sysbios_knl_Swi_Object__get__S
0084ce20   ti_sysbios_knl_Task_Object__get__S
0084ce80   ti_sysbios_knl_Task_allBlockedFunction__I
0084cee0   ti_sysbios_knl_Task_enter__I
0084cf40   vsprintf
0084cfa0   writemsg
0084cff8   C$$IO$$
0084d000   xdc_runtime_Memory_calloc__F
0084d060   xdc_runtime_SysStd_abort__F
0084d0c0   xdc_runtime_System_aprintf_va__F
0084d0c0   xdc_runtime_System_avprintf__F
0084d120   xdc_runtime_System_printf_va__F
0084d120   xdc_runtime_System_vprintf__F
0084d180   xdc_runtime_Text_cordText__F
0084d1e0   PHYREG_read
0084d220   __c6xabi_isinf
0084d2a0   _args_main
0084d320   ti_sysbios_family_c62_TaskSupport_buildTaskStack
0084d360   ti_sysbios_family_xxx_Hwi_switchToIsrStack
0084d3e0   free
0084d520   strlen
0084d560   ti_sysbios_BIOS_startFunc__I
0084d5a0   ti_sysbios_BIOS_start__E
0084d5e0   ti_sysbios_family_c64p_Hwi_Module__startupDone__F
0084d620   ti_sysbios_family_c64p_Hwi_Object__delete__S
0084d660   ti_sysbios_family_c64p_Hwi_disableInterrupt__E
0084d6a0   ti_sysbios_family_c64p_Hwi_enableInterrupt__E
0084d6e0   ti_sysbios_gates_GateHwi_Handle__label__S
0084d720   ti_sysbios_gates_GateHwi_Object__delete__S
0084d760   ti_sysbios_gates_GateMutex_Handle__label__S
0084d7a0   ti_sysbios_gates_GateMutex_Instance_finalize__F
0084d7e0   ti_sysbios_gates_GateMutex_Object__delete__S
0084d820   ti_sysbios_gates_GateMutex_leave__E
0084d860   ti_sysbios_hal_Hwi_HwiProxy_Object__create__S
0084d8a0   ti_sysbios_hal_Hwi_Instance_finalize__F
0084d8e0   ti_sysbios_hal_Hwi_Params__init__S
0084d920   ti_sysbios_hal_Timer_Module__startupDone__F
0084d960   ti_sysbios_heaps_HeapMem_Handle__label__S
0084d9a0   ti_sysbios_heaps_HeapMem_Object__delete__S
0084d9e0   ti_sysbios_knl_Clock_Object__destruct__S
0084da20   ti_sysbios_knl_Clock_Params__init__S
0084da60   ti_sysbios_knl_Queue_Object__destruct__S
0084daa0   ti_sysbios_knl_Semaphore_Instance_finalize__F
0084dae0   ti_sysbios_knl_Semaphore_Object__destruct__S
0084db20   ti_sysbios_knl_Task_Object__first__S
0084db60   ti_sysbios_knl_Task_Object__next__S
0084dba0   ti_sysbios_knl_Task_Params__init__S
0084dbe0   ti_sysbios_timers_timer64_Timer_Module__startupDone__F
0084dc20   xdc_runtime_Error_check__F
0084dc60   xdc_runtime_Error_init__F
0084dca0   xdc_runtime_Error_raiseX__E
0084dce0   xdc_runtime_Gate_leaveSystem__F
0084dda0   xdc_runtime_Memory_free__F
0084dde0   xdc_runtime_Registry_findById__F
0084de20   xdc_runtime_Startup_exec__I
0084de60   xdc_runtime_System_abort__F
0084dea0   xdc_runtime_System_aprintf__E
0084dee0   xdc_runtime_System_printf__E
0084df20   xdc_runtime_Text_ropeText__F
0084df60   xdc_runtime_Text_visitRope__I
0084dfa0   CSL_GPIO_open
0084dfc0   MDIO_getStatus
0084e000   MDIO_initPHY
0084e040   __c6xabi_negll
0084e060   __cxa_atexit
0084e080   __cxa_ia64_exit
0084e0a0   __xdc__init
0084e0c0   _nop
0084e140   _register_lock
0084e160   _register_unlock
0084e180   ti_sysbios_family_c62_TaskSupport_glue
0084e1a0   ti_sysbios_family_xxx_Hwi_switchToTaskStack
0084e1c0   C$$EXIT
0084e1c0   abort
0084e1e0   atexit
0084e200   __TI_decompress_none
0084e220   __TI_decompress_rle24
0084e240   emac_get_version
0084e280   putc
0084e2a0   putchar
0084e2c0   ti_sysbios_BIOS_RtsGateProxy_enter__E
0084e2e0   ti_sysbios_BIOS_RtsGateProxy_leave__E
0084e300   ti_sysbios_BIOS_setThreadType__E
0084e320   ti_sysbios_family_c62_TaskSupport_Module__startupDone__S
0084e340   ti_sysbios_family_c62_TaskSupport_checkStack__E
0084e360   ti_sysbios_family_c62_TaskSupport_getStackAlignment__E
0084e380   ti_sysbios_family_c64p_Exception_Module_startup__E
0084e3a0   ti_sysbios_family_c64p_Hwi_Module__startupDone__S
0084e3c0   ti_sysbios_family_c64p_Hwi_Module_startup__E
0084e3e0   ti_sysbios_family_c64p_Hwi_clearInterrupt__E
0084e400   ti_sysbios_family_c64p_Hwi_startup__E
0084e420   ti_sysbios_family_c64p_Hwi_switchFromBootStack__E
0084e440   ti_sysbios_family_c64p_Hwi_unPluggedInterrupt__I
0084e460   ti_sysbios_family_c64p_tci6488_TimerSupport_enable__E
0084e480   ti_sysbios_family_c66_Cache_Module_startup__E
0084e4a0   ti_sysbios_family_c66_Cache_wbInv__E
0084e4c0   ti_sysbios_gates_GateHwi_Instance_init__F
0084e4e0   ti_sysbios_gates_GateHwi_enter__E
0084e500   ti_sysbios_gates_GateHwi_leave__E
0084e520   ti_sysbios_gates_GateHwi_query__E
0084e540   ti_sysbios_gates_GateHwi_query__F
0084e560   ti_sysbios_gates_GateMutex_query__E
0084e580   ti_sysbios_gates_GateMutex_query__F
0084e5a0   ti_sysbios_hal_Hwi_HwiProxy_Module__startupDone__S
0084e5c0   ti_sysbios_hal_Hwi_HwiProxy_Object__delete__S
0084e5e0   ti_sysbios_hal_Hwi_HwiProxy_clearInterrupt__E
0084e5e0   ti_sysbios_hal_Hwi_clearInterrupt__E
0084e600   ti_sysbios_hal_Hwi_HwiProxy_disableInterrupt__E
0084e600   ti_sysbios_hal_Hwi_disableInterrupt__E
0084e620   ti_sysbios_hal_Hwi_HwiProxy_enableInterrupt__E
0084e620   ti_sysbios_hal_Hwi_enableInterrupt__E
0084e640   ti_sysbios_hal_Hwi_HwiProxy_startup__E
0084e640   ti_sysbios_hal_Hwi_startup__E
0084e660   ti_sysbios_hal_Hwi_HwiProxy_switchFromBootStack__E
0084e660   ti_sysbios_hal_Hwi_switchFromBootStack__E
0084e680   ti_sysbios_hal_Hwi_Module_startup__E
0084e6a0   ti_sysbios_hal_Hwi_Module_startup__F
0084e6c0   ti_sysbios_hal_Timer_Module__startupDone__S
0084e6e0   ti_sysbios_hal_Timer_Module_startup__E
0084e700   ti_sysbios_hal_Timer_Module_startup__F
0084e720   ti_sysbios_hal_Timer_TimerProxy_Module__startupDone__S
0084e740   ti_sysbios_hal_Timer_TimerProxy_getExpiredCounts__E
0084e760   ti_sysbios_hal_Timer_TimerProxy_getPeriod__E
0084e780   ti_sysbios_hal_Timer_TimerProxy_setNextTick__E
0084e7a0   ti_sysbios_hal_Timer_TimerProxy_startup__E
0084e7a0   ti_sysbios_hal_Timer_startup__E
0084e7c0   ti_sysbios_heaps_HeapMem_Module_GateProxy_enter__E
0084e7e0   ti_sysbios_heaps_HeapMem_Module_GateProxy_leave__E
0084e800   ti_sysbios_heaps_HeapMem_Module_GateProxy_query__E
0084e820   ti_sysbios_heaps_HeapMem_isBlocking__E
0084e860   ti_sysbios_knl_Clock_Module_startup__E
0084e880   ti_sysbios_knl_Queue_Instance_init__F
0084e8a0   ti_sysbios_knl_Queue_empty__E
0084e8c0   ti_sysbios_knl_Swi_Module_startup__E
0084e8e0   ti_sysbios_knl_Swi_disable__E
0084e900   ti_sysbios_knl_Task_Module_startup__E
0084e920   ti_sysbios_knl_Task_SupportProxy_Module__startupDone__S
0084e940   ti_sysbios_knl_Task_SupportProxy_checkStack__E
0084e960   ti_sysbios_knl_Task_SupportProxy_getStackAlignment__E
0084e980   ti_sysbios_knl_Task_SupportProxy_start__E
0084e9a0   ti_sysbios_knl_Task_SupportProxy_swap__E
0084e9c0   ti_sysbios_knl_Task_disable__E
0084e9e0   ti_sysbios_timers_timer64_Timer_Module__startupDone__S
0084ea00   ti_sysbios_timers_timer64_Timer_Module_startup__E
0084ea20   ti_sysbios_timers_timer64_Timer_TimerSupportProxy_enable__E
0084ea40   ti_sysbios_timers_timer64_Timer_setNextTick__E
0084ea80   xdc_runtime_Error_check__E
0084eaa0   xdc_runtime_Error_init__E
0084eac0   xdc_runtime_Error_print__E
0084eae0   xdc_runtime_Gate_enterSystem__E
0084eb00   xdc_runtime_Gate_enterSystem__F
0084eb20   xdc_runtime_Gate_leaveSystem__E
0084eb40   xdc_runtime_Memory_HeapProxy_alloc__E
0084eb60   xdc_runtime_Memory_HeapProxy_free__E
0084eb80   xdc_runtime_Memory_alloc__E
0084eba0   xdc_runtime_Memory_calloc__E
0084ebc0   xdc_runtime_Memory_free__E
0084ebe0   xdc_runtime_Registry_findById__E
0084ec00   xdc_runtime_Startup_exec__E
0084ec20   xdc_runtime_Startup_reset__I
0084ec40   xdc_runtime_SysStd_abort__E
0084ec60   xdc_runtime_SysStd_exit__E
0084ec80   xdc_runtime_SysStd_exit__F
0084eca0   xdc_runtime_SysStd_putch__E
0084ecc0   xdc_runtime_SysStd_putch__F
0084ece0   xdc_runtime_SysStd_ready__E
0084ed00   xdc_runtime_SysStd_ready__F
0084ed20   xdc_runtime_System_Module_GateProxy_enter__E
0084ed40   xdc_runtime_System_Module_GateProxy_leave__E
0084ed60   xdc_runtime_System_Module_startup__E
0084ed80   xdc_runtime_System_Module_startup__F
0084eda0   xdc_runtime_System_SupportProxy_abort__E
0084edc0   xdc_runtime_System_SupportProxy_exit__E
0084ede0   xdc_runtime_System_SupportProxy_putch__E
0084ee00   xdc_runtime_System_SupportProxy_ready__E
0084ee20   xdc_runtime_System_abort__E
0084ee40   xdc_runtime_System_atexit__E
0084ee60   xdc_runtime_System_exit__E
0084ee80   xdc_runtime_System_exit__F
0084eea0   xdc_runtime_System_lastFxn__I
0084eec0   xdc_runtime_System_vsprintf__E
0084eee0   xdc_runtime_System_sprintf_va__F
0084eee0   xdc_runtime_System_vsprintf__F
0084ef00   xdc_runtime_Text_cordText__E
0084ef20   xdc_runtime_Text_putLab__E
0084ef40   xdc_runtime_Text_putSite__E
0084ef60   xdc_runtime_Text_ropeText__E
0084ef80   ti_sysbios_heaps_HeapMem_Instance_State_0_buf__A
00856f80   xdc_runtime_Text_charTab__A
00859228   ti_sysbios_family_c66_Cache_marvalues__C
00859628   _ctypes_
00859730   xdc_runtime_Text_nodeTab__A
0085993c   ti_sysbios_knl_Task_Object__PARAMS__C
00859974   ti_sysbios_family_c64p_Hwi_Object__PARAMS__C
008599a4   ti_sysbios_BIOS_Module__diagsEnabled__C
008599a8   emac_version_str
00859a04   ti_sysbios_hal_Hwi_Object__PARAMS__C
00859a80   ti_sysbios_heaps_HeapMem_Module__FXNS__C
00859aa8   xdc_runtime_Startup_sfxnTab__A
00859ad0   ti_sysbios_gates_GateHwi_Module__FXNS__C
00859af4   ti_sysbios_gates_GateMutex_Module__FXNS__C
00859b18   ti_sysbios_knl_Clock_Object__PARAMS__C
00859b3c   ti_sysbios_knl_Semaphore_Object__PARAMS__C
00859ba4   ti_sysbios_family_c64p_Hwi_Object__DESC__C
00859bc4   ti_sysbios_gates_GateHwi_Object__DESC__C
00859be4   ti_sysbios_gates_GateMutex_Object__DESC__C
00859c04   ti_sysbios_hal_Hwi_Object__DESC__C
00859c24   ti_sysbios_heaps_HeapMem_Object__DESC__C
00859c44   ti_sysbios_heaps_HeapMem_Object__PARAMS__C
00859c64   ti_sysbios_knl_Clock_Object__DESC__C
00859c84   ti_sysbios_knl_Queue_Object__DESC__C
00859ca4   ti_sysbios_knl_Semaphore_Object__DESC__C
00859cc4   ti_sysbios_knl_Task_Object__DESC__C
00859ce4   ti_sysbios_BIOS_Module__diagsIncluded__C
00859d00   ti_sysbios_gates_GateHwi_Object__PARAMS__C
00859d18   ti_sysbios_gates_GateMutex_Object__PARAMS__C
00859d30   ti_sysbios_knl_Queue_Object__PARAMS__C
00859d48   ti_sysbios_knl_Task_hooks__A
00859d60   xdc_runtime_Startup_sfxnRts__A
00859d74   ti_sysbios_family_c66_Cache_initSize__C
00859d94   ti_sysbios_BIOS_Module__diagsMask__C
00859d98   xdc_runtime_Startup_firstFxns__A
00859dac   ti_sysbios_knl_Idle_funcList__C
00859db4   ti_sysbios_knl_Task_hooks__C
00859dbc   xdc_runtime_Startup_firstFxns__C
00859dc4   xdc_runtime_Startup_lastFxns__C
00859dcc   ti_sysbios_BIOS_installedErrorHook__C
00859dd8   ti_sysbios_family_c62_TaskSupport_stackAlignment__C
00859ddc   ti_sysbios_family_c64p_Exception_E_exceptionMin__C
00859de0   ti_sysbios_family_c64p_Exception_exceptionHook__C
00859de4   ti_sysbios_family_c64p_Exception_externalHook__C
00859de8   ti_sysbios_family_c64p_Exception_internalHook__C
00859dec   ti_sysbios_family_c64p_Exception_nmiHook__C
00859df0   ti_sysbios_family_c64p_Hwi_E_alreadyDefined__C
00859df4   ti_sysbios_family_c64p_Hwi_E_handleNotFound__C
00859df8   ti_sysbios_family_c64p_Hwi_LD_end__C
00859dfc   ti_sysbios_family_c64p_Hwi_LM_begin__C
00859e00   ti_sysbios_family_c64p_Hwi_Module__diagsEnabled__C
00859e04   ti_sysbios_family_c64p_Hwi_Module__diagsIncluded__C
00859e08   ti_sysbios_family_c64p_Hwi_Module__diagsMask__C
00859e0c   ti_sysbios_family_c64p_Hwi_Module__loggerFxn1__C
00859e10   ti_sysbios_family_c64p_Hwi_Module__loggerFxn8__C
00859e14   ti_sysbios_family_c64p_Hwi_Module__loggerObj__C
00859e18   ti_sysbios_family_c66_Cache_atomicBlockSize__C
00859e1c   ti_sysbios_gates_GateMutex_A_badContext__C
00859e20   ti_sysbios_gates_GateMutex_Instance_State_sem__O
00859e24   ti_sysbios_gates_GateMutex_Module__diagsEnabled__C
00859e28   ti_sysbios_gates_GateMutex_Module__diagsIncluded__C
00859e2c   ti_sysbios_gates_GateMutex_Module__diagsMask__C
00859e30   ti_sysbios_hal_Hwi_E_stackOverflow__C
00859e34   ti_sysbios_heaps_HeapMem_A_align__C
00859e38   ti_sysbios_heaps_HeapMem_A_heapSize__C
00859e3c   ti_sysbios_heaps_HeapMem_A_invalidFree__C
00859e40   ti_sysbios_heaps_HeapMem_A_zeroBlock__C
00859e44   ti_sysbios_heaps_HeapMem_E_memory__C
00859e48   ti_sysbios_heaps_HeapMem_Module__diagsEnabled__C
00859e4c   ti_sysbios_heaps_HeapMem_Module__diagsIncluded__C
00859e50   ti_sysbios_heaps_HeapMem_Module__diagsMask__C
00859e54   ti_sysbios_heaps_HeapMem_Module__gateObj__C
00859e58   ti_sysbios_heaps_HeapMem_Object__count__C
00859e5c   ti_sysbios_heaps_HeapMem_Object__table__C
00859e60   ti_sysbios_heaps_HeapMem_reqAlignMask__C
00859e64   ti_sysbios_heaps_HeapMem_reqAlign__C
00859e68   ti_sysbios_knl_Clock_A_badThreadType__C
00859e6c   ti_sysbios_knl_Clock_LM_begin__C
00859e70   ti_sysbios_knl_Clock_LM_tick__C
00859e74   ti_sysbios_knl_Clock_LW_delayed__C
00859e78   ti_sysbios_knl_Clock_Module_State_clockQ__O
00859e7c   ti_sysbios_knl_Clock_Module__diagsEnabled__C
00859e80   ti_sysbios_knl_Clock_Module__diagsIncluded__C
00859e84   ti_sysbios_knl_Clock_Module__diagsMask__C
00859e88   ti_sysbios_knl_Clock_Module__loggerFxn1__C
00859e8c   ti_sysbios_knl_Clock_Module__loggerFxn2__C
00859e90   ti_sysbios_knl_Clock_Module__loggerObj__C
00859e94   ti_sysbios_knl_Clock_tickMode__C
00859e98   ti_sysbios_knl_Clock_tickSource__C
00859e9c   ti_sysbios_knl_Queue_Object__count__C
00859ea0   ti_sysbios_knl_Idle_funcList__A
00859ea4   ti_sysbios_knl_Queue_Object__table__C
00859ea8   ti_sysbios_knl_Semaphore_A_badContext__C
00859eac   ti_sysbios_knl_Semaphore_A_noEvents__C
00859eb0   ti_sysbios_knl_Semaphore_A_overflow__C
00859eb4   ti_sysbios_knl_Semaphore_Instance_State_pendQ__O
00859eb8   ti_sysbios_knl_Semaphore_LM_pend__C
00859ebc   ti_sysbios_knl_Semaphore_LM_post__C
00859ec0   ti_sysbios_knl_Semaphore_Module__diagsEnabled__C
00859ec4   ti_sysbios_knl_Semaphore_Module__diagsIncluded__C
00859ec8   ti_sysbios_knl_Semaphore_Module__diagsMask__C
00859ecc   ti_sysbios_knl_Semaphore_Module__loggerFxn2__C
00859ed0   ti_sysbios_knl_Semaphore_Module__loggerFxn4__C
00859ed4   ti_sysbios_knl_Semaphore_Module__loggerObj__C
00859ed8   ti_sysbios_knl_Swi_LD_end__C
00859edc   ti_sysbios_knl_Swi_LM_begin__C
00859ee0   ti_sysbios_knl_Swi_LM_post__C
00859ee4   ti_sysbios_knl_Swi_Module__diagsEnabled__C
00859ee8   ti_sysbios_knl_Swi_Module__diagsIncluded__C
00859eec   ti_sysbios_knl_Swi_Module__diagsMask__C
00859ef0   ti_sysbios_knl_Swi_Module__loggerFxn1__C
00859ef4   ti_sysbios_knl_Swi_Module__loggerFxn4__C
00859ef8   ti_sysbios_knl_Swi_Module__loggerObj__C
00859efc   ti_sysbios_knl_Swi_Object__count__C
00859f00   ti_sysbios_knl_Swi_Object__table__C
00859f04   ti_sysbios_knl_Task_A_badPriority__C
00859f08   ti_sysbios_knl_Task_A_badTaskState__C
00859f0c   ti_sysbios_knl_Task_A_badThreadType__C
00859f10   ti_sysbios_knl_Task_A_noPendElem__C
00859f14   ti_sysbios_knl_Task_E_spOutOfBounds__C
00859f18   ti_sysbios_knl_Task_E_stackOverflow__C
00859f1c   ti_sysbios_knl_Task_LD_block__C
00859f20   ti_sysbios_knl_Task_LD_exit__C
00859f24   ti_sysbios_knl_Task_LD_ready__C
00859f28   ti_sysbios_knl_Task_LM_switch__C
00859f2c   ti_sysbios_knl_Task_Module_State_inactiveQ__O
00859f30   ti_sysbios_knl_Task_Module_State_terminatedQ__O
00859f34   ti_sysbios_knl_Task_Module__diagsEnabled__C
00859f38   ti_sysbios_knl_Task_Module__diagsIncluded__C
00859f3c   ti_sysbios_knl_Task_Module__diagsMask__C
00859f40   ti_sysbios_knl_Task_Module__loggerFxn2__C
00859f44   ti_sysbios_knl_Task_Module__loggerFxn4__C
00859f48   ti_sysbios_knl_Task_Module__loggerObj__C
00859f4c   ti_sysbios_knl_Task_Object__count__C
00859f50   ti_sysbios_knl_Task_Object__heap__C
00859f54   ti_sysbios_knl_Task_Object__table__C
00859f58   ti_sysbios_knl_Task_allBlockedFunc__C
00859f5c   ti_sysbios_knl_Task_defaultStackHeap__C
00859f60   ti_sysbios_knl_Task_defaultStackSize__C
00859f64   ti_sysbios_knl_Task_numConstructedTasks__C
00859f68   ti_sysbios_knl_Task_numPriorities__C
00859f6c   ti_sysbios_timers_timer64_Timer_A_notAvailable__C
00859f70   ti_sysbios_timers_timer64_Timer_E_cannotSupport__C
00859f74   ti_sysbios_timers_timer64_Timer_Module__diagsEnabled__C
00859f78   ti_sysbios_timers_timer64_Timer_Module__diagsIncluded__C
00859f7c   ti_sysbios_timers_timer64_Timer_Module__diagsMask__C
00859f80   ti_sysbios_timers_timer64_Timer_anyMask__C
00859f84   ti_sysbios_timers_timer64_Timer_freqDivisor__C
00859f88   ti_sysbios_timers_timer64_Timer_numLocalTimers__C
00859f8c   ti_sysbios_timers_timer64_Timer_numTimerDevices__C
00859f90   xdc_runtime_Assert_E_assertFailed__C
00859f94   xdc_runtime_Core_A_initializedParams__C
00859f98   xdc_runtime_Core_Module__diagsEnabled__C
00859f9c   xdc_runtime_Core_Module__diagsIncluded__C
00859fa0   xdc_runtime_Core_Module__diagsMask__C
00859fa4   xdc_runtime_Error_E_generic__C
00859fa8   xdc_runtime_Error_E_memory__C
00859fac   xdc_runtime_Error_Module__diagsEnabled__C
00859fb0   xdc_runtime_Error_Module__diagsIncluded__C
00859fb4   xdc_runtime_Error_Module__diagsMask__C
00859fb8   xdc_runtime_Error_Module__loggerFxn8__C
00859fbc   xdc_runtime_Error_Module__loggerObj__C
00859fc0   xdc_runtime_Error_policy__C
00859fc4   xdc_runtime_Error_raiseHook__C
00859fc8   xdc_runtime_IGateProvider_Interface__BASE__C
00859fcc   xdc_runtime_IHeap_Interface__BASE__C
00859fd0   xdc_runtime_IModule_Interface__BASE__C
00859fd4   xdc_runtime_Log_L_error__C
00859fd8   xdc_runtime_Memory_defaultHeapInstance__C
00859fdc   xdc_runtime_Startup_execImpl__C
00859fe0   xdc_runtime_Startup_lastFxns__A
00859fe4   xdc_runtime_Startup_maxPasses__C
00859fe8   xdc_runtime_Startup_sfxnRts__C
00859fec   xdc_runtime_Startup_sfxnTab__C
00859ff0   xdc_runtime_Startup_startModsFxn__C
00859ff4   xdc_runtime_System_Module__gateObj__C
00859ff8   xdc_runtime_System_extendFxn__C
00859ffc   xdc_runtime_System_maxAtexitHandlers__C
0085a000   xdc_runtime_Text_charTab__C
0085a004   xdc_runtime_Text_nameEmpty__C
0085a008   xdc_runtime_Text_nameStatic__C
0085a00c   xdc_runtime_Text_nameUnknown__C
0085a010   xdc_runtime_Text_nodeTab__C
0085a014   xdc_runtime_Text_visitRopeFxn__C
0085a018   ti_sysbios_BIOS_Module__id__C
0085a01c   ti_sysbios_family_c64p_Exception_Module__id__C
0085a020   ti_sysbios_family_c64p_Hwi_Module__id__C
0085a024   ti_sysbios_family_c64p_Hwi_Module__loggerDefined__C
0085a028   ti_sysbios_gates_GateMutex_Module__id__C
0085a02c   ti_sysbios_hal_Hwi_Module__id__C
0085a030   ti_sysbios_heaps_HeapMem_Module__id__C
0085a034   ti_sysbios_knl_Clock_Module__id__C
0085a038   ti_sysbios_knl_Clock_Module__loggerDefined__C
0085a03c   ti_sysbios_knl_Semaphore_Module__id__C
0085a040   ti_sysbios_knl_Semaphore_Module__loggerDefined__C
0085a044   ti_sysbios_knl_Swi_Module__id__C
0085a048   ti_sysbios_knl_Swi_Module__loggerDefined__C
0085a04c   ti_sysbios_knl_Task_Module__id__C
0085a050   ti_sysbios_knl_Task_Module__loggerDefined__C
0085a054   ti_sysbios_knl_Task_deleteTerminatedTasks__C
0085a058   ti_sysbios_knl_Task_initStackFlag__C
0085a05c   ti_sysbios_timers_timer64_Timer_Module__id__C
0085a060   ti_sysbios_timers_timer64_Timer_startupNeeded__C
0085a064   xdc_runtime_Core_Module__id__C
0085a068   xdc_runtime_Error_Module__loggerDefined__C
0085a06c   xdc_runtime_Error_maxDepth__C
0085a070   xdc_runtime_Memory_Module__id__C
0085a074   xdc_runtime_Text_charCnt__C
0085a078   xdc_runtime_Text_isLoaded__C
0085a07c   xdc_runtime_Text_registryModsLastId__C
0085a080   xdc_runtime_Text_unnamedModsLastId__C
0085a088   emac_mcb
0085ba8c   app_mcb
0085d1c8   _tmpnams
0085d308   gI2cBlock
0085d358   ti_sysbios_knl_Task_Instance_State_0_hookEnv__A
0085d360   _stack
0085e360   __TI_STACK_END
0085e360   _ftable
0085e540   ti_sysbios_BIOS_Module__state__V
0085e55c   ti_sysbios_family_c64p_Exception_Module__state__V
0085e588   ti_sysbios_family_c64p_Hwi_Module__root__V
0085e590   ti_sysbios_family_c64p_Hwi_Module__state__V
0085e5f8   ti_sysbios_gates_GateHwi_Module__root__V
0085e600   ti_sysbios_gates_GateMutex_Module__root__V
0085e608   ti_sysbios_hal_Hwi_Module__root__V
0085e610   ti_sysbios_hal_Timer_Module__root__V
0085e618   ti_sysbios_heaps_HeapMem_Module__root__V
0085e620   ti_sysbios_knl_Clock_Module__root__V
0085e628   ti_sysbios_knl_Clock_Module__state__V
0085e654   ti_sysbios_knl_Queue_Module__root__V
0085e65c   ti_sysbios_knl_Semaphore_Module__root__V
0085e664   ti_sysbios_knl_Swi_Module__root__V
0085e66c   ti_sysbios_knl_Swi_Module__state__V
0085e688   ti_sysbios_knl_Task_Module__root__V
0085e690   ti_sysbios_knl_Task_Module__state__V
0085e6c4   ti_sysbios_timers_timer64_Timer_Module__root__V
0085e6cc   ti_sysbios_timers_timer64_Timer_Module__state__V
0085e6e0   xdc_runtime_Error_Module__state__V
0085e6e4   xdc_runtime_Memory_Module__state__V
0085e6e8   xdc_runtime_Registry_Module__state__V
0085e6f0   xdc_runtime_Startup_Module__state__V
0085e6f8   xdc_runtime_System_Module__state__V
0085e704   xdc_runtime_Text_Module__state__V
0085e70c   __xdc__init__addr
0085e710   ti_sysbios_timers_timer64_Timer_Module_State_0_device__A
0085e870   ti_sysbios_knl_Swi_Module_State_0_readyQ__A
0085e8f0   ti_sysbios_knl_Task_Module_State_0_readyQ__A
0085e9e8   ti_sysbios_timers_timer64_Timer_Object__table__V
0085ea34   _ft_end
0085ea38   TSK_idle
0085ea38   ti_sysbios_knl_Task_Object__table__V
0085ea80   ti_sysbios_gates_GateMutex_Object__table__V
0085eac0   ti_sysbios_timers_timer64_Timer_Module_State_0_gctrl__A
0085eb00   ti_sysbios_timers_timer64_Timer_Module_State_0_handles__A
0085eb40   ti_sysbios_timers_timer64_Timer_Module_State_0_intFreqs__A
0085eb80   ti_sysbios_knl_Swi_Object__table__V
0085ebb0   ti_sysbios_knl_Clock_Object__table__V
0085ebd0   xdc_runtime_System_Module_State_0_atexitHandlers__A
0085ec08   ti_sysbios_family_c64p_Hwi_Object__table__V
0085ec20   ti_sysbios_heaps_HeapMem_Object__table__V
0085ec34   _cleanup_ptr
0085ec38   _dtors_ptr
0085ec3c   __TI_enable_exit_profile_output
0085ec40   _lock
0085ec44   _unlock
0085ec48   ti_sysbios_hal_Hwi_Object__table__V
0085ec50   ti_sysbios_hal_Timer_Object__table__V
0085ec58   ti_sysbios_gates_GateHwi_Object__table__V
0085ec60   ti_sysbios_knl_Task_Instance_State_0_stack__A
0085f480   emac_comm_dev0
0085f600   emac_comm_pcb0
0085f614   __CIOBUF_
0085f7a4   __TI_STATIC_BASE
0085f7a4   hGpio
0085f7ac   platform_errno
0085f7b0   platform_init_return_code
0085f7b4   pktbuf_extmem
0085f800   ti_sysbios_family_c64p_Hwi0
0085f820   ti_sysbios_family_c64p_Hwi1
0085f840   ti_sysbios_family_c64p_Hwi2
0085f860   ti_sysbios_family_c64p_Hwi3
0085f880   ti_sysbios_family_c64p_Hwi4
0085f8a0   ti_sysbios_family_c64p_Hwi5
0085f8c0   ti_sysbios_family_c64p_Hwi6
0085f8e0   ti_sysbios_family_c64p_Hwi7
0085f900   ti_sysbios_family_c64p_Hwi8
0085f920   ti_sysbios_family_c64p_Hwi9
0085f940   ti_sysbios_family_c64p_Hwi10
0085f960   ti_sysbios_family_c64p_Hwi11
0085f980   ti_sysbios_family_c64p_Hwi12
0085f9a0   ti_sysbios_family_c64p_Hwi13
0085f9c0   ti_sysbios_family_c64p_Hwi14
0085f9e0   ti_sysbios_family_c64p_Hwi15
0085ff20   __TI_Handler_Table_Base
0085ff2c   __TI_Handler_Table_Limit
0085ff5c   __TI_CINIT_Base
0085ffa4   __TI_CINIT_Limit
80000898   gDeviceNandBBlist
80000cb4   gDeviceNand
80000cec   gDeviceNor
80000d24   gDeviceEeprom0
80000d5c   gDeviceEeprom1
80000d98   emac_port_mode
ffffffff   __TI_pprof_out_hndl
ffffffff   __TI_prof_data_size
ffffffff   __TI_prof_data_start
ffffffff   __binit__
ffffffff   __c_args__
ffffffff   binit
UNDEFED    __TI_INITARRAY_Base
UNDEFED    __TI_INITARRAY_Limit

[803 symbols]
